:020000041102E7
:10000000F0B502230124514E514D8FB000203370C2
:100010002C7005F04FFE07F0A3FB07F0EFFD07F093
:10002000D7FA1F2200214B4B0EAF1A704A4B1C709F
:100030004A4B19704A4B19689143163A0A431A60A1
:10004000602219689143403A0A431A6007F060FA47
:1000500007F026FCC120FF21424B80001A588A433A
:100060001A50C522920098588843BF3901439950CD
:1000700098583D4908408021C9010143802099508A
:100080009958C0050902090A01439950802137484F
:10009000490107F0E5FB0323220035490194009351
:1000A000344807F075FB2C22334903A807F098FA6F
:1000B00003AC61782078023405F08CFBA742F8D1BC
:1000C0002E4B2F4A19682F4C1140A022D2020A430E
:1000D0001A608022196892040A431A6019682A4A31
:1000E0001140802292030A431A60284B284A934207
:1000F00024D9032007F094FA2368264A88331A602B
:1001000007F07EFB07F08CF9307807F0F1F92878DA
:10011000C0B207F0CDF807F0CBFA1F49042007F072
:100120005FFB05F093FD02211C4807F061F800F029
:10013000B1F800F019FA00200FB0F0BD012007F06F
:100140006FFA2368164A8833D9E7C0464A0AFF1F68
:10015000BC44FF1F480AFF1F490AFF1F680AFF1F10
:10016000BCF0004000E100E0FF00FFFFC044FF1FC3
:100170004457FF1FC054FF1FD078021114F00040F5
:10018000FF7FF8FF7464FF1FFFFF9FFF7C6BFF1F63
:10019000FF7BFF1F00C0FF1F3B00010800C00311D1
:1001A0000080FF1F70B500252C492D4A2D484D6356
:1001B00008CA1B051B0DED188242F9D100222A4BFB
:1001C0002A4C8B632A4B1A6280222A4B9205DA67EB
:1001D0000822E3689343E360274B1B78012B03D08D
:1001E000A368264A1340A3600021072005F01CFBEA
:1001F0000021072005F0D8FB0021072005F0EAFACE
:100200000122E36811209343E360EE24E4006C4391
:1002100007F03EFA112007F05BF8112007F030FAE2
:10022000174A200C0400642390420AD8FA220023C3
:10023000D200904205D9134B0A21C01807F000FBE9
:10024000C3B2114A1372114BD4801B78002B04D116
:100250000F4B1021187807F0FBF970BD0000054026
:100260008805054000060540FF0100003CF0004005
:1002700000F0004004E100E04A0AFF1FFFDFFFFF3B
:10028000B70B000030F8FFFFE061FF1FEE63FF1FB8
:10029000EA61FF1F002210B51100112007F0E8FAF3
:1002A00010BD0000F8B5002301250826374F384C53
:1002B0003B62E3681120AB43E360E368B343E36070
:1002C00007F006F8112007F0E3F9112007F0F8F81D
:1002D0004023226800211343236080236268DB02ED
:1002E000134363608023A26807201343A360A368BD
:1002F000284A1340A3608023A2689B011343102265
:10030000A360236C93432364236C2B4323648023D7
:100310005B003B62226B204B1A402263626B1A40E7
:100320006263A26B1A40A263E26B1340E3631B4A51
:10033000E3681340E36005F04DFA2900072005F05B
:1003400037FA2900072005F06FFA112007F038F876
:10035000134B144AC72013608023626B5B03134363
:100360006363E36880003343E360E3680E4A1D4340
:100370000E4BE56019581140802212020A431A50B0
:10038000802292051A600A4B5E63F8BD00F00040BF
:100390003CF00040FFFFDFFFEFFFEFFFFFFF7FFFBD
:1003A000A5010211F403FF1FFF00FFFF00E100E0C1
:1003B0000000054030B503A804880B20002C0ED1A6
:1003C0004968074D08784978090201430A20A94283
:1003D00005D1012120001980024B1B7A137030BD1A
:1003E000192A0000E061FF1FF7B5150008AA16885A
:1003F0004A680F4F14785278120222430A24BA42F4
:1004000014D10122DBB2019200962A0006F06CFBA7
:10041000041E0BD1074B1B68002B07D068782A7885
:100420000002104342425041013098472000FEBD77
:1004300002290000C461FF1F30B5012503790400C3
:10044000BFB02B4212D00A49408805F0B9FE2842BD
:100450000CD06A46074B69465B8D55801380064B6E
:1004600060881B7A1371002202F05EFF3FB030BD3E
:10047000BC61FF1F8841FF1FE061FF1F10B50549E8
:10048000054805F053FE0421044A054805F010FE16
:1004900010BDC046BC61FF1FFFFF0000FC780211C9
:1004A0008841FF1F10B5024803F0C4FD10BDC046CF
:1004B000390402110623837010330371443B4371E6
:1004C0002A3383714433C37100230222012110B502
:1004D00003720E4B027041701C8881724472197A4B
:1004E0000273C1729A784273DA7882730322C273FC
:1004F0001A7902745A7942740C2282749A79C274FD
:10050000DB7903751123C37010BDC046E061FF1F86
:1005100010B5142006F05CFF124B14220021186065
:1005200006F0AEFF002006F0BBFF012006F088FFBA
:10053000022006F08DFF032003F020F8042005F0D0
:1005400035F8052002F06EFA062002F02BFF072096
:1005500000F05AFC082005F08BFD092000F070FA2D
:1005600010BDC046C861FF1F10B506F0F1FF0120A5
:1005700006F07EFF06F00CFF002010BD70B51600DF
:1005800004AA148805AA15784A68507811780002E0
:100590002A4A0843801805284BD806F031FF031378
:1005A0001E29343F0720032C0BD80422121BAA4219
:1005B00000D92A0022491A803000091906F0D8FF14
:1005C000002070BD07200F2CFBD81022121BAA425E
:1005D00000D92A001B491A80EEE707200E2CF0D81C
:1005E0000F22121BAA4200D92A0017491A80E3E7FA
:1005F0000720032CE5D80422121BAA4200D92A00A6
:1006000012491A80D8E70720032CDAD80422121BDB
:10061000AA4200D92A000E491A80CDE70720032CF0
:10062000CFD80422121BAA4200D92A0009491A80F5
:10063000C2E700220A201A80C3E7C046DCD5FFFFCC
:100640006B790211CC61FF1F5B790211567902119F
:10065000517902114C79021110B50D21024A03485B
:1006600005F026FD10BDC04640790211CC41FF1FA8
:1006700010B500210D2005F003FA01210C2005F032
:10068000FFF906F00DFE0400092006F019FF002214
:10069000184BDA6661321A6019685B3A9143023A84
:1006A0000A431A60144A944209D10A22DA610732D5
:1006B0001A6200221A639A630132DA6310BD0F4A8C
:1006C000944203D11E22DA610532F1E70C4A9442CA
:1006D00003D13022DA610632EAE70A4A944203D1B2
:1006E0004322DA610832E3E7074A9442E1D1692202
:1006F000F7E7C046005000400024F4000048E8013D
:10070000006CDC020090D00300D8B80510B50024BE
:10071000064B0920DC6606F0DBFD21000D2005F00C
:1007200043F921000C2005F03FF910BD00500040B6
:10073000F8B51C000023134D0F00EB66686016002F
:1007400007F02EF801238022EB6623002F61520070
:10075000013B08D207F064F808200B4A1168002C0E
:1007600003D12000F8BD2A61F2E72B6F034203D0CA
:100770002B69013C3370013613685B1A0A2BEED9E2
:100780000124EEE7005000406008FF1F002370B511
:100790000C4C0D00E366606007F002F80123E3668D
:1007A000256107F03DF88020074A80001168636BDF
:1007B000034205D113685B1A0A2BF8D9012070BDDA
:1007C0000020FCE7005000406008FF1F002370B5C8
:1007D000134C0E00E3666060150006F0E1FF012394
:1007E000E36626610F33626B1A42FCD02B0A236149
:1007F0001023626B1A42FCD0EDB2256107F010F8AD
:100800008020084A80001168636B034205D1136899
:100810005B1A0A2BF8D9012070BD0020FCE7C04606
:10082000005000406008FF1F13B5FFF721FF0223AF
:10083000002101AA4020FFF77BFF6A460400022343
:10084000012140200632FFF773FF0443FFF75EFFEC
:10085000002C1CD16B469A880F4BD2BA53430F48D9
:100860000F491B181B144B806B46DA880D4B52BA8C
:100870005204520C53430C4A1B181B0C934200D1D8
:100880000A4B8B800B8801330B80200016BD07F0CC
:1008900073F90124F9E7C04606640000FF7F0000F9
:1008A000E061FF1F204E0000102700000F2700000E
:1008B00070470000013870B5042809D806F0A0FD83
:1008C000030920081200134B0221187806F0C0FE1D
:1008D00070BD104B0821187806F0EAFF00220E4B7D
:1008E0001A70F5E700240B4D0C4B082128780C4AB0
:1008F0001C7006F005FE2100287806F031FDE7E7C0
:100900000122064B08211A70024B187806F0D0FF1E
:10091000DEE7C046EA61FF1FEC61FF1FEB61FF1FCE
:100920001027000010B5002902D1112005F06CF845
:1009300010BD000010B5084B084C9881D881188272
:100940005882207801F00CFF0422054B0121207809
:100950001A7006F07DFE10BD6643FF1F1E64FF1F68
:100960001D64FF1F10B501290CD11322064B112065
:100970001A7005F049F8054B1B78002B02D004488B
:10098000FFF7D8FF10BDC046EB61FF1FEE63FF1FEE
:10099000C40900000300F0B50A4D8E18B14202D11F
:1009A00052008018F0BD0C782F6824093C5D0F2799
:1009B0001C700C7801313C402F683C5D5C70023348
:1009C000ECE7C046AC42FF1F10B5064A06490420BA
:1009D00005F01CF9112005F003F90121112005F0A3
:1009E00013F810BD250902116509021110B5114B4C
:1009F0001A781870002A0ED000280BD10E4B1A78E6
:100A0000062A07D85423D340DB0703D50B4B1878AD
:100A100001F0A6FE10BD0028FCD0074B1B78012B6F
:100A200002D0033B022BF5D8044B0121187806F0C5
:100A30000FFEEFE7EE63FF1F1D64FF1F1E64FF1F25
:100A4000F0B5554D85B02870FFF7BEFF07F094F85C
:100A500006F056FC002002A90290039006F060FD0B
:100A600003224E494E48FFF795FF2D240300022232
:100A70001C704C490130FFF78DFF0222047002A95F
:100A80000130FFF787FF0222474B484CDA872000EE
:100A900006F0D6FD022816D006222100444802ABFB
:100AA00006F050FA00280ED00321200006F0F0FED8
:100AB0008D23E3706E3B23710622193321003C48DD
:100AC000637106F0F3FA0D233A4F3B4C3B4E3B70FB
:100AD000013B23700422033B3000394963700196C7
:100AE00006F046FD2D23012236493748A371FFF752
:100AF00051FF01223549FFF74DFF01222B49FFF736
:100B000049FF0020FFF772FF314E324A0121324B7C
:100B10001278307801F0E6FD3A78012723000021B1
:100B2000307801F0DFFD21782C4B0139019AC9B2F0
:100B300000201F7005F0DAF9FA221B4B52019A814E
:100B4000DA811A825A822021287806F071FE01206B
:100B5000404205F017FA0120404205F0B3FAFFF7D2
:100B60007BFDFFF78BFC00F061FC380006F078FCA1
:100B7000380006F02DFEF72000F070FF39002878CD
:100B800006F066FD287801F047FF154806F0E0FB07
:100B9000FFF788FB05B0F0BDEA61FF1FDC43FF1FD4
:100BA000CC61FF1FDE61FF1F6643FF1F6509FF1F4A
:100BB000ADAC0000EA63FF1FCB63FF1FCD63FF1FD7
:100BC0006B7902116709FF1FD263FF1F6609FF1FC0
:100BD0001E64FF1FE042FF1FC142FF1FBC63FF1FD7
:100BE000EE61FF1F20230A0070B51A400D00194264
:100BF0002DD03B4B1B78002B20D03A4A0121137893
:100C00000133DBB21800137008400B4219D0FFF714
:100C10000BFE354C2000FFF74DFC2100152006F09F
:100C200067FD324A1378002B08D0013BDBB213700A
:100C3000002B03D1FA204001FFF77CFE2020684002
:100C400070BD232BFAD91070FFF72CFBF6E70BB21F
:100C5000002B0ADA264B187806F0B2FD002801D0E6
:100C600006F0BEFB80200002E9E702240E002640C9
:100C7000214206D01B4B01201A70FFF7B7FE20005F
:100C8000DDE70B0710D5FFF7CFFD00F0E9FB154AB4
:100C900013780133DBB2052B02D813700820CEE79E
:100CA0001670FFF7FFFAF9E71024214206D00C4B2B
:100CB0001B78002BE3D1FFF7F5FBE0E7012421428D
:100CC00005D00C4800F064F806F042FDD7E7042395
:100CD000080018401942B3D04B401800B0E7C04696
:100CE000EE63FF1FEC61FF1FC142FF1FEB61FF1F9F
:100CF000EA61FF1FA442FF1FF0B51B4B1B4F1B886F
:100D00003A8804001A4E1B4D85B09A420DD832889D
:100D10009A420AD3184B1A882B889A4205D1174A4F
:100D2000174B12881B889A421BD0052000F0ECFE5E
:100D30003B8802AA13803388019053802B88114D81
:100D400093800F4B02A91B88D3800F4B2A781888F9
:100D500002F0F8FB0D4B08212878019A1C7006F070
:100D6000E7FC05B0F0BDC046BA63FF1FB642FF1FE7
:100D7000B442FF1FB242FF1FB863FF1FB663FF1FDD
:100D8000B042FF1F1E64FF1FB842FF1FB463FF1F66
:100D900013B50C4B1C78002C11D1002801D00A4B44
:100DA00018600A4A0A4B11780A4A10780A4A0192D6
:100DB0000A4A0092002204F091FF200016BD11247F
:100DC000FBE7C0461D64FF1FB063FF1F1C64FF1FCD
:100DD0000C64FF1F1E64FF1FF863FF1FFC63FF1FEF
:100DE00010B5064B12201B78052B06D1044B13229D
:100DF0001988044B187801F063F810BD1D64FF1FBB
:100E0000B842FF1F1E64FF1F10B500240122114BC2
:100E100052421870104B1C70104B1A8001F0FCFDF0
:100E200004220F4B21001A700E480C3206F028FBEA
:100E3000102221000C4806F023FB07220B4B1C60FC
:100E40000B4B1C700B4B1C700B4B1A700B4B1C701C
:100E500010BDC0461E64FF1F1D64FF1FB842FF1F68
:100E60001C64FF1F0C64FF1FFC63FF1FF863FF1F60
:100E7000CA63FF1FC963FF1FBA42FF1FC863FF1F7A
:100E8000F8B5174C0600257806A814240078052D1F
:100E900023D1B41F134FA5B21824BD421DD88D1FF6
:100EA000ADB2BD4219D8FA256D00AA4215D21D0077
:100EB0000D4F0A3DADB2BD420FD80C4C26800C4CF4
:100EC00021800C4900240A800B4A1380FFF714FF8D
:100ED0000A4B0421187806F0EBFC2000F8BDC04650
:100EE0001D64FF1F790C0000750C0000B642FF1F47
:100EF000B442FF1FB242FF1FB042FF1F1E64FF1F1C
:100F0000F0B50BB20D0089B0002B00DB76E1A64EE8
:100F1000307806F055FC041E55D00378A22B00D182
:100F200027E1D02B1AD0912B4AD143780E2B47D1F1
:100F30009E4B82889A4243D19D4A83681278052A43
:100F40003ED1032018567F283AD09A4B1B68002BBD
:100F500036D05B68002B33D0984731E08078072883
:100F60002ED806F04DFA042D1D444479ADDD63788A
:100F7000002B11D10622E11C8F4806F0F9FA01215D
:100F80008B4B19708D4B1A78002A5BD08C4B3078C4
:100F900001F0A8FB002855D00722854B1A7051E0BC
:100FA00061780029F8D1E378002B11D0854A864B6F
:100FB0001278307801F096FB60706378002BEBD1EB
:100FC000200006F00DFA80200002684009B0F0BD54
:100FD000774B1B78022BF3D00121307806F0E8FA2A
:100FE0000028EAD10121307806F032FBE5E763788A
:100FF000002BD1D16E4F032807D13B78052B02D1AE
:1010000001333B701EE00223FBE7704B1A88704BE4
:101010000293002A0BD01B78002B03D001213078DB
:1010200006F086FB3B78062B04D1013BE9E7029BE7
:101030001A70F7E7042B41D10121029B3078197017
:1010400006F006FB5B4B1B68002BB9D01B68002B1E
:10105000B6D0574A10787FE76378554F002B27D1D9
:101060000622211D5B4806F083FA62895A4B5B49D0
:101070001A80A2895A4B1A80E3890B8005213970A6
:1010800058490A80584A1380228A584B1A80584B74
:101090001B78012B09D11F2000F036FDFA229200A7
:1010A00042430421307806F043FB0022484B75E7A9
:1010B000312B00D070E70022454B1A700323A0E7C4
:1010C00006220021434806F0DBF90023454A0421AB
:1010D0001380454A30781380444A138006F0E8FBB9
:1010E0000821307806F0E4FBA379083B5A425341CB
:1010F0002F4A03331370314B1B78002B06D0344B2F
:1011000030781A78002A06D001F02AFB0122324BEF
:1011100052421A8096E70121197006F099FAF5E714
:101120000821307806F0C4FB6378002B00D047E735
:101130002C4B2E4F0293E388029A042113802A4BF2
:10114000307803932389039A138063893B8006F0E8
:101150002FFA002800D033E7264B1B68002B00D164
:101160002EE7039902983A88098800881B689847F7
:1011700026E74379132B00D022E70389012B0AD1FC
:101180001D4B1B78022B06D10821307806F090FB0E
:10119000FFF726FE14E7052000F0B6FC0821020048
:1011A000307806F0C5FA0BE71E64FF1F0514000037
:1011B0001D64FF1FB063FF1FEF63FF1FE042FF1FAF
:1011C000C142FF1FEA63FF1FCB63FF1FEC63FF1FDA
:1011D000EE63FF1FBD63FF1FB842FF1FC463FF1F05
:1011E000C663FF1FBA63FF1FB863FF1FB663FF1F0D
:1011F000BC63FF1FAC63FF1FB463FF1F8020C001EF
:10120000014200D0E1E6CB0731D5324B1B78002BF1
:101210001DD0314E05AC3378052B1AD1023B23701B
:101220002E4B21001B7823722D4B1B7863722D4BA4
:10123000187801F0FBF9002809D007202A4B3070FC
:101240001B68002B03D01B68002B00D0984701209F
:10125000BBE60E20254B06221B7825492370254B23
:101260001B78637002ABC01806F082F9D8E702233E
:1012700008001840194209D0174B1B78052B03D1E1
:101280001D4B188806F0C4FA02209EE60424214271
:1012900003D0FFF731FD200097E60823080018402F
:1012A000194200D192E6154B1C78012C03D0022C78
:1012B0000DD0082089E6124B124A134913481B88A7
:1012C0001288098800880094FFF7DAFDF1E7FFF73C
:1012D00087FDEEE7EE63FF1F1D64FF1FBA42FF1F8D
:1012E000C863FF1F1E64FF1FB063FF1FCA63FF1F99
:1012F000BB42FF1FC963FF1FB842FF1FB463FF1F3C
:10130000B042FF1FB242FF1FB442FF1FB642FF1F91
:1013100010B502A804880B20002C10D14968087869
:101320004978090201430C48814209D10221198000
:101330000A4B59881170DB7800205BB2537010BDE6
:10134000074C0A20A142FAD102211980034B998847
:1013500011705B79F0E7C0466E2A0000E061FF1F64
:101360006F2A0000F7B5150008AA16884A680F4FC3
:1013700014785278120222430A24BA4214D101226C
:10138000DBB2019200962A0005F0AEFB041E0BD1E1
:10139000074B1B68002B07D068782A78000210439F
:1013A00042425041013098472000FEBD0229000012
:1013B0003064FF1F30B5012503790400BFB02B4214
:1013C00027D01549408804F0FBFE28420DD06A461C
:1013D000124B69465B8D138002235380104B5B8850
:1013E00093806088002201F09FFF0E49608804F01E
:1013F000E7FEC0070DD56A460B4B69461B88138074
:1014000002235380064B9B8893806088002201F062
:101410008BFF3FB030BDC0462864FF1FE442FF1F72
:10142000E061FF1F2064FF1F3E43FF1F10B5074C04
:101430000749200004F07AFE2000064904F076FEF9
:101440000721054A054804F033FE10BDFFFF0000E8
:101450002864FF1F2064FF1FFC790211E442FF1F74
:1014600010B5024802F0E6FD10BDC046B5130211EA
:1014700010B5034C0B000122210000F06BFA10BDE7
:10148000311602110B8870B506000D000224162BD0
:1014900011D92B000322094900F05CFA041E0AD17D
:1014A000074B2A881B88191C934200D9111C300055
:1014B00089B200F0EFFA200070BDC0465D1602113F
:1014C0008E64FF1F10B54A780400013A0B00022019
:1014D000012A07D80A78002A04D0052220000249F0
:1014E00000F038FA10BDC0468B1602110A7810B50C
:1014F0000B0004000220002A04D007222000024929
:1015000000F028FA10BDC046371702110A7810B54E
:101510000B0004000220002A04D009222000024906
:1015200000F018FA10BDC0469D17021110B5034C0B
:101530000B000B22210000F00DFA10BDCD17021197
:1015400010B5034C0B000D22210000F003FA10BD72
:101550003F18021110B5034C0B000F22210000F0C0
:10156000F9F910BD991802110A7810B50B000400A2
:101570000220002A04D011222000024900F0EAF9DA
:1015800010BDC046A9180211002310B5132219007E
:1015900000F0E0F910BD000010B5034C0B0017225D
:1015A000210000F0D7F910BDFB180211002310B57F
:1015B0001922190000F0CEF910BD000010B5034C3F
:1015C0000B001B22210000F0C5F910BD35190211D6
:1015D000F7B584890D0006000121002C22D00023DC
:1015E0008268D3561778002B1EDA0C2C1AD90C3CC3
:1015F000A4B2131940880093230002F076FE431E24
:10160000984101307B06DB0F6B703F23013C1F408C
:10161000A4B22870AF70AC80002C07D0B36801333F
:10162000AB6000210800FEBD0020EBE7AC60F8E7EE
:101630000B7803704B8843704B881B0A83700B79BF
:10164000C370042070470420022B06D10020537879
:1016500011781B02009A0B43138070470B880370AC
:101660000B881B0A437002207047042000998342B4
:101670000AD1537810781B0203430B80D3789078FB
:101680001B02034300204B807047F8B50D004B78D8
:1016900001240021461C03702B788B4201D82000C6
:1016A000F8BD6B78B01C4F1C012B10D18900691854
:1016B0004B88022233704B88B9001B0A737069187B
:1016C00005F056FF04360434A4B2F9B2E4E712235D
:1016D00059436B185A88043132705B8810221B0AF8
:1016E0007370691805F044FF12361234ECE770B5D8
:1016F000049D14001E00052B01D8042070BD6378E2
:1017000012781B0213432B80E378A2781B02134349
:1017100002226B802A71211D681D063E05F028FFFC
:10172000B2B22A81F02AE8D82800A11D0A3005F0BB
:101730001FFF0020E2E7002310B50A789A4201D883
:10174000900010BD9A008A185488013304705488A0
:10175000DBB2240A4470948884709288120AC270A2
:101760000430EAE710B51100029C062B04D00420D7
:101770001022142B01D010BD022222714B78087860
:101780001B0203432380CB7888781B0203436380CA
:101790000431601D05F0ECFE0020ECE710B50C787C
:1017A0008B7804315C43E4B203702200013005F011
:1017B000DFFE601C10BD0420022B06D100205378F0
:1017C00011781B02009A0B431380704710B50C0070
:1017D0000A88023105F0CCFE208810BD70B50400E7
:1017E0000D0004981100012B01D8042070BD16785B
:1017F00052781202324302800200F832557014709F
:10180000E825002C00D10C35023B9AB24280AA4256
:10181000EBD80231043005F0ABFE0020E6E70420EF
:10182000009983420AD1537810781B0203430B803E
:10183000D37890781B02034300204B80704710B58B
:101840000C000A88023105F093FE208810BD0000CC
:1018500070B501211E000420049C0E400B4218D1DB
:10186000CB40DDB28D4214D90A49DBB209889942D6
:101870000FD32300F6331D70330058001118497838
:10188000165C0902314301332152D9B28D42F4D89A
:10189000002070BD6043FF1F10B50C000A880231A4
:1018A00005F066FE208810BD10B50C788B780431E9
:1018B0005C43E4B203702200013005F059FE601C65
:1018C00010BD10B511000298032B01D8042010BDE3
:1018D00014785278043B120222430280CA788C7832
:1018E0001202224342809AB28280F22AEED8043158
:1018F000063005F03DFE0020E9E710B50C000B882E
:1019000003700B881B0A43704B8883704B881B0A3B
:10191000C3708A880430063105F02AFEA08804309E
:1019200080B210BD0420012B03D100201378009A4F
:101930001370704710B50C000B8803700B881B0ADE
:1019400043704A880230043105F012FE608802308C
:1019500080B210BDF0B589B003931E4B02924200D5
:101960000700D05A019102F010F81325061E2DD061
:10197000029B01240370019B002B04D000190399E2
:101980009847001984B26B461B7A5BB2002B0FDAC2
:101990001021380002F00CFB1925002813D130006B
:1019A0003219E1B202F056FC051E0CD10C34A4B27F
:1019B000042304AA380005A993800696948101F0B7
:1019C0009FFD051E02D0300005F0E2FD280009B0A1
:1019D000F0BDC0468C64FF1F70B505000C000028E8
:1019E0000CD00020814209D010222000044905F0CB
:1019F000BFFD01202B7823736B78637370BDC046E5
:101A0000167A0211F0B506000D0017001C0085B013
:101A100002291BD00020102907D1022B07D0102B40
:101A200003D115E00020102C08D005B0F0BD6946A8
:101A30003800FFF7D1FF2A0069460BE06946300005
:101A4000FFF7CAFF22006946380004E0022BE9D103
:101A50002A003900300005F01BFDE6E7031CF728DB
:101A600000D9F723032008499AB2013A0B80D31713
:101A7000034006499B189B100B80D30F04499B1809
:101A80005B100B807047C0466443FF1F6243FF1F1B
:101A90006043FF1F034B1B888B4202D3024B400065
:101AA000C15270476443FF1F8C64FF1F014B40000D
:101AB000185A70478C64FF1F1722014B1A80704719
:101AC0008C64FF1F70B505000E2005F039FE041E62
:101AD00013D0D0230370002306228370074945707A
:101AE000033005F045FD064B2100DA8A62811B7E3A
:101AF0002373044B187805F07BFE70BDA864FF1FAC
:101B00009864FF1FB443FF1F262803D8024B4000F0
:101B1000C05A70470148FCE76643FF1FFFFF000003
:101B200070B506000C00094D1C220021280005F0AC
:101B3000A7FC074B1E70074B1C7005F079FD0123B5
:101B4000002801D0002312202B7070BD9864FF1F65
:101B5000B443FF1FB964FF1F70B505000D4C0800AA
:101B6000E260A16010220021656005F0D1FD01282E
:101B700003D11021A06802F048FD102200212800A6
:101B800005F0C6FD012803D11021606802F03DFD7B
:101B900070BDC0469864FF1F70B5041E05D10029B2
:101BA00003D006220D4805F0E3FC0D4B1D78012DF6
:101BB00011D1002C05D102221A7005F0B9FC2800C1
:101BC00070BD00221A70074B1B78FF2BF7D0200046
:101BD000FFF778FFF3E70025F1E7C046A864FF1F91
:101BE0009864FF1FB443FF1F030010B5002801D104
:101BF000002010BD00780B4A002803D15988D182FB
:101C00001B7913761378022BF2D10023984200D16E
:101C100003331370044B1B78FF2B01D0FFF752FFE7
:101C20000120E6E79864FF1FB443FF1F002911D08D
:101C300000280CD04B79012803D140225242134393
:101C400003E03F221340032802D001204B7170476C
:101C50004022F4E70800FAE770B5094D0100287842
:101C600000280BD0074C0622200005F081FC210043
:101C70002878FFF7DBFF200005F0CAFB70BDC046E7
:101C8000B864FF1F9264FF1F00290AD0012808D101
:101C90003F224B799343C02B03D0403B5A425341E0
:101CA000981C704770B5174D06002B78FF2B15D088
:101CB0000A2005F045FD041E10D0D0230370C83B58
:101CC0008370114B11491B784670C3700622043093
:101CD00005F04EFC2100287805F08AFD0C4B1B789E
:101CE000012B0DD10B4B1B68002B03D09B68002BE5
:101CF00000D09847084B04211878084A05F000FCEA
:101D000070BDC046B443FF1FB864FF1F9264FF1F3D
:101D1000B464FF1FE064FF1FE464FF1F60EA00007B
:101D2000014B98687047C0469864FF1F014BDB6801
:101D3000186870479864FF1F074B10B5DA6813687E
:101D400001331360054B1878FF2803D08021C901A7
:101D500005F07EFC10BDC0469864FF1FB443FF1F12
:101D6000F7B50E0002F0B8F8051E1CD00E4B066247
:101D70001F78002F00D10778AB791020019305F070
:101D8000DFFC041E0FD0D0230380C73B8370019B70
:101D9000E91DC3700622043005F0EAFB210038007B
:101DA000E66005F025FDF7BDB243FF1F014B187833
:101DB0007047C046B864FF1F054B002805D1054B8E
:101DC0001A78054B002A00D1014B18007047C04615
:101DD000A864FF1FB864FF1F9264FF1F014B58687F
:101DE0007047C0469864FF1F024B1868431E984115
:101DF000C0B27047BC64FF1F421E03000120152AB9
:101E000003D9FF3B5A425341D8B27047F0B51C008A
:101E100000230E0085B0039002920B70029A934249
:101E200001D3002019E0E55C5A1CD2B2002DF8D095
:101E3000029851198142F4DC0233DFB2A35C18002E
:101E40000193FFF7D9FF002807D0013D019A0399BC
:101E5000EBB233708A4202D1E01905B0F0BDDB1954
:101E6000DBB2DBE710B50C0002F08EF803001220A5
:101E7000002B03D02100588805F0F2FB10BD0000B4
:101E800070B50E4D84006359002B15D0186A0028D8
:101E900001D005F0EDFB2B59586A002801D005F060
:101EA000E7FB2B59986A002801D005F0E1FB28597F
:101EB00005F0DEFB00232B5170BDC046C864FF1F38
:101EC0001C4B70B504000E00150099420AD11A4B44
:101ED0001B68002B01D1122070BD1B68002BFAD0AB
:101EE0009847F9E7154B994215D1134B1B68002B06
:101EF0000AD01B68002B07D09847002804D1104B4C
:101F00001C70104B1D70E7E729002000FFF7AAFFA7
:101F10000028E1D1F3E7080001F0DEFF0028DAD065
:101F200003780320A342D7D12900300005F098FBA5
:101F3000D2E7C046FEFF0000C464FF1FFFFF0000A1
:101F4000C164FF1FC064FF1FF7B50400808801F063
:101F5000C3FF0025A84203D00578A08801F0F8FF50
:101F60001C4E3378002B1FD0AB421DD11A4B2800DA
:101F70001978FFF777FF002818D000233370A37972
:101F80000820A778A688019305F0DAFB011E0DD082
:101F9000D0230370CA3B8370019B47708680837196
:101FA000280005F025FC01E0002DE8D1A0880B4BAE
:101FB0008200D358002B01D0FFF762FF1721A088C1
:101FC000FFF768FDA08801F017FDA08801F0EEFD85
:101FD000F7BDC046C164FF1FC064FF1FC864FF1F78
:101FE000F0B587B01D000CAB1B88070001930DAB4B
:101FF0001B88142002930EAB1B88160003930FABB3
:102000001B880091049310AB1B88059305F098FB87
:10201000041E1AD0D0230370CB3B47708370C67068
:10202000062229000430002D11D005F0A1FA019BF1
:1020300021006381029B0098A381039BE381049BA1
:102040002382059BA37405F0D3FB07B0F0BD05F018
:1020500017FAECE7F7B5009308AB1B8807000C20D4
:102060000D001600019305F06BFB041E13D0280031
:1020700001F032FF00280FD00078D0232370C93B35
:10208000A370009B21002381019B6770A580E680DF
:10209000638105F0ADFBF7BD014B1878EDE7C04655
:1020A000B443FF1F13B5040064890389C288818883
:1020B000C0780094FFF7CEFF13BD000010B5044CAC
:1020C0002068002803D005F0D3FA0023236010BD58
:1020D000CC64FF1FA122F0B5818892004A43384B9F
:1020E000384F1B6804009B189D2292009B18827930
:1020F00089B01A603B68002B5FD01D78324B1B689B
:10210000002B04D05B68002B01D0002098472600EC
:1021100008363100E079FFF7B7FD237DE07102005A
:10212000E0780493638A29000393238A0293E38966
:102130000193A38800933300FFF752FFE378002B4D
:102140000BD1E289A379A18802920196E279280055
:102150000092012201F0CAFEE0703B68002B20D003
:10216000FFF7ACFF194D287800281AD0184B1978C2
:10217000FFF778FE002814D02B78E6780820079324
:10218000A78805F0DDFA011E09D0D0230370CA3BF1
:102190004670837087808671079805F029FB0023BD
:1021A0002B701721A088FFF775FCA08801F024FC94
:1021B000A08801F0FBFC09B0F0BD064B9DE7C046CE
:1021C0003409FF1FCC64FF1FE064FF1FC164FF1FC1
:1021D000C064FF1FB443FF1FF8B5070008000E00DE
:1021E00001F07AFE041E18D02620FFF78DFC051E94
:1021F00000D12578062005F0A3FA041E0DD0002199
:10220000062205F03DF9D0232370C23B2100677000
:10221000A370A680E8B205F0EBFAF8BDF0B585B082
:1022200001930AAB1B78070002930BAB1B780800E5
:102230000D000092039301F04FFE061E22D01020E5
:1022400005F07EFA041E1DD01022002105F018F9B9
:102250002620FFF759FC002800D13078D0232370C6
:10226000C13BA370009B21002372019B67706372C6
:10227000029BA580A372039BC0B2E3720C9BE36038
:1022800005F0B6FA05B0F0BDF7B50D00019001F00C
:1022900023FE071E20D00E2005F052FA041E1BD08C
:1022A0002620FFF731FC061E00D13E78D023238084
:1022B000C53B0622A370F91DE01C05F059F9019BEE
:1022C0002A0063810123DD401A401D402100227352
:1022D0006573F0B205F08CFAF7BD0000F0B585B07B
:1022E000029010000D0017000A9E039301F0F4FD08
:1022F000041E31D0029B002B2ED1039B02795B0779
:1023000024D5122313430422002E08D10B9900294F
:1023100005D10C99002902D10D9900291AD01A4330
:102320000D9B2271002B00D0C9E0002E00D1CFE020
:10233000002D00D0CCE0606A002801D005F098F9AB
:102340001C21300005F0C4F9606205E002239A43C5
:102350000E33D7E793432371654BBA00D458002C52
:1023600000D1AAE0002E10D0236A002B03D11C203C
:1023700005F02EF820625E4BBA00D358186A002888
:1023800003D01C22310005F0F3F80C9B002B12D077
:10239000574CBB001D596B6A002B03D1162005F06A
:1023A00017F86862BB00E358586A002803D0162269
:1023B0000C9905F0DDF80D9B002B11D04C4DBC00A5
:1023C0006659B36A002B03D1142005F001F8B062FE
:1023D0002B59986A002803D014220D9905F0C8F8EB
:1023E000380001F079FD051E67D0414BBA00D35883
:1023F000002B62D01A6A3420002A00D11C389A6A55
:10240000002A01D0143080B20B9A002A01D01C306F
:1024100080B25B6A002B01D0163080B205F090F9D3
:10242000041E4AD01822002105F02AF82620FFF7C2
:102430006BFB0190002801D12B780193D0232370EE
:10244000029B200063700A23294EA370039BBD00EA
:10245000A371AB59A780196A1830002905D01C2236
:10246000A06005F085F8200034307359996A00297E
:1024700007D0030014221433E060029305F078F8CB
:1024800002980B9B002B08D003001C221C330B99D5
:102490002061029305F06CF802987359596A00297B
:1024A00003D01622606105F063F86B4621001879AD
:1024B00005F09EF93800FFF7E3FC05B0F0BD1022EF
:1024C0000D9B0D991B69A018236205F051F82CE7AC
:1024D0000B9B002B00D13FE7012D00D03CE7606A49
:1024E000002801D005F0C4F81C210B982AE7C0464B
:1024F000C864FF1F10B5044C2068002803D005F005
:10250000B7F80023236010BDBC64FF1F0B4B07B559
:102510001A68002A01D100200EBD6946531C012013
:1025200012780731FFF772FC0028F4D002780123FB
:10253000100018401A42EED0EEE7C046D864FF1FE4
:10254000F0B51F4F01203B6887B0002B25D09B784A
:10255000059300F0B3FB002821D00A20FFF7D4FA3E
:1025600004000B20FFF7D0FA164B05001E78731EEF
:102570009E413B68F6B2191DD878FFF757FB3B68C0
:102580002900DA7A043303929A7901930292009037
:1025900033002000059A04F02BFF07B0F0BDFFF7D1
:1025A000B5FF002805D00620FFF7AEFA040007208B
:1025B000D8E70820FFF7A8FA04000920D2E7C046B0
:1025C000BC64FF1FB864FF1F70B50A4E0400337867
:1025D0000D00FF2B0DD0042005F0B2F8011E08D02D
:1025E000D0230370CE3B45708370C470307805F003
:1025F000FFF870BDC443FF1F70B5040006200D0036
:1026000005F09EF8011E0AD0D0230370CD3B8370E5
:10261000054B44701B688580187805F0E9F8002C9C
:1026200001D0FFF767FF70BDBC64FF1FF8B5264FF0
:1026300006003B680D001124002B05D10522234B19
:102640001B78134202D112242000F8BD204A102426
:102650001268002AF8D01278002AF5D0DB0719D5C5
:102660002B789A1E012A1AD80C2004F0B1FE1324EC
:1026700038600028E8D000230A2243702900067041
:10268000023004F075FFFFF75BFF041E0AD0FFF76E
:1026900031FFD9E700F012FB0028E1D1E4E7002B7D
:1026A000E2D0D0E70B4B1B78032BCDD11D20FFF7D9
:1026B0002BFA094B18800028C6D0084B0421187843
:1026C000074A04F01DFFBFE7BC64FF1FB964FF1F8A
:1026D000D864FF1FB864FF1FB664FF1FE464FF1FC8
:1026E00060EA0000F7B50193194B14001A7805232E
:1026F00006000F0012201A4221D0012920D1154BCB
:102700001D68002D1BD002201F2C18D8002C02D0D1
:10271000019B002B13D0104B1F221E706E1C00213A
:10272000300004F0ADFE01992200300004F020FFDB
:10273000310020002C70002F06D004F039FEFEBDC1
:10274000064B12201D68DCE705F0BAF8F7E7C04633
:10275000B964FF1FD864FF1FC443FF1FD464FF1F69
:10276000F8B50F4E12243368002B17D01B780F3C9E
:10277000834213D100250B4F0221387805F098F8D9
:10278000094B042138781D8005F092F8074B28008A
:102790001D8033685C7005F00BF804002000F8BD64
:1027A000BC64FF1FE464FF1FD064FF1FB664FF1FFB
:1027B00070B5012823D11B4C2388002B03D01A4A63
:1027C0001578002D07D0194B1B68002B02D0187804
:1027D000FFF7C6FF70BD3B2B02D93C3B2380F9E7D6
:1027E000134E0221307805F063F8FA222388920014
:1027F00002215A43307804F09BFF2580EAE70B4B17
:102800001B68002BE6D00B4B1B785B07E2D5084B0F
:102810000221187805F04CF80022024B1A80FFF7CD
:1028200069FED7E7D064FF1FB464FF1FBC64FF1FBD
:10283000E464FF1FB964FF1FF8B51E4D2868002827
:1028400003D004F015FF00232B601B4E30680028D6
:1028500003D004F00DFF00233360184F05243B78AC
:1028600018002040234221D0154800F02BFA3B7875
:10287000234213D0202004F0ABFD2860002813D0A1
:102880002022002104F0FCFD202004F0A1FD041E04
:10289000306005D02022002104F0F2FD002004E089
:1028A000286804F0E5FE2C601320F8BD00F00AFA59
:1028B000F4E7C046D864FF1FD464FF1FB964FF1F4C
:1028C000B843FF1F10B50A4C23681A1E0ED000280B
:1028D00008D10130587004F06BFF002805D0236840
:1028E000002B02D00021FFF787FE0122100010BD4F
:1028F000BC64FF1FF7B5274E050033680191181E11
:1029000021D05C78244F012C30D1FFF7FFFD002847
:1029100025D02000FFF7F8F80400412814D91F4BF8
:10292000022118781E4A04F0EBFD1E4B3C3C1C8033
:10293000022233685A703B78002B14D12800019989
:10294000FFF75AFE0120FEBDFA2292004243002A00
:10295000EED0124B0221187804F0EAFEE8E7FFF708
:10296000D3F80200F3E700233B70EBE73B78002B42
:10297000E8D1032004F0E4FE011E08D0D023037048
:10298000CC3B457083703368187804F031FFFFF753
:10299000B1FDD7E7BC64FF1FB464FF1FE464FF1FF1
:1029A00060EA0000D064FF1F10B517498388020059
:1029B0008B4220D011D815498B4217D014490020E2
:1029C0005B1899B2012907D8926811785A4253418D
:1029D000D8B2FFF7F9FD012010BD0E4A00209B1868
:1029E00007229BB29A424041C0B2F5E7836818784B
:1029F000FFF768FFF0E7836899785A78090218783A
:102A00001143FFF777FFE7E70A20000006200000E8
:102A1000F8DFFFFFAFDFFFFF014B18707047C046C4
:102A2000C543FF1F10B5064C207001F031FA207825
:102A300004F056FC0521207800F052FD10BDC04680
:102A4000E464FF1F0BB273B50D00002B00DBC4E084
:102A5000884B187804F0B4FE041E0ED00378912B36
:102A60000FD0A22B00D1A1E0834B1878FF2852D0C1
:102A7000210004F0BDFE00284DD1802000026840F6
:102A800076BD43780F2B76D013D8052B70D00E2B44
:102A9000EAD18088794B98422BD8794B98421BD841
:102AA000784B9842E0D1A3681878591CFFF774F866
:102AB00038E03E2BD8D18378032B74D06CD8012B0F
:102AC0006ED0022BD0D1704B1B68002B23D05B68DB
:102AD000002B20D098471EE06C4BC0180C28C3D8A0
:102AE00004F01EFC1DC2C2150BC20B0B0B3223C21D
:102AF0003C00674BC0180728B6D8664B1B68002BF4
:102B000009D01B68002B06D0200098470AE0A36874
:102B10001878FFF7C7F8200004F062FCADE7A06862
:102B2000FFF762F800289FD0F5E7A3681B78002B19
:102B3000F1D0554B1B68002BEDD01B68002BEAD061
:102B4000210055489847EDE74F4B1B68002BE2D01A
:102B50001B68002BDFD021005048F3E7504B1B6867
:102B6000002BD8D05B68002BD5D021004348E9E783
:102B7000FFF7EAF9CFE780884A4B984203D04A4BE7
:102B8000984200D070E7464B1B68002BC3D05B68AF
:102B9000002BC0D02100D5E7153B012BBBD963E743
:102BA000FFF798FAB7E7FFF77DFAB4E73F4B1B78DA
:102BB000042B07D100236A4613800179408800F076
:102BC000B5FCA8E7364B1B68002BA4D05B68002B34
:102BD000A1D00100364898479DE7012421420AD040
:102BE000294B1B68002B04D05B68002B01D0002010
:102BF0009847012043E78B070AD5264B1B68002B1B
:102C000004D05B68002B01D020009847022036E7F3
:102C10000421280008400D4200D131E7254E3388B9
:102C2000002B21D0013B9BB23380002B1AD1FFF740
:102C3000DBF800280AD0204B1C70164B1B68002BB9
:102C400004D05B68002B01D020009847FFF7C6F83E
:102C5000694601F0F1FC6846FEF7FEFF1D20FEF715
:102C600053FF308004200AE7024B187804F020FE5E
:102C7000F8E7C046E464FF1FC543FF1F0E200000B5
:102C80000120000009100000DC64FF1FFEDFFFFFD1
:102C9000AFDFFFFFE064FF1F0C2000000B200000EF
:102CA000C464FF1F0D20000013200000B964FF1F43
:102CB000FFFF0000B664FF1FB464FF1F10B501F0F2
:102CC0008BF910BD014B18607047C046E064FF1FD0
:102CD0000B880020162B01D817230420014A1380EB
:102CE0007047C0468E64FF1F00207047074A0300EC
:102CF0001188814207D091880020994202D1013089
:102D00008000101870470020FAE7C046EC64FF1FEF
:102D1000F0B58F7806000D00C7B01E2F15D1FFF754
:102D2000E5FF051E03D10024200047B0F0BD0022BE
:102D30003B003100C078009200F0A2FB0400A81C08
:102D400000F0C3FBFF23EB70EEE7264B0624039352
:102D50001B78FF2BE8D0182FE6D87B08224A013BCE
:102D6000DB0002929A589446002ADDD0029AD318CA
:102D70005B68002BD8D00878002802D14B78012B53
:102D800002D10624122FCFD107AFAB886978009704
:102D90006446AA68A047041EC6D1AB78029A5B08B5
:102DA000013BDB00D318390030005B689847041EF4
:102DB0000BD1AB78042BB6D0039A310010782200E7
:102DC000009700F05DFB0400AEE76A78002AABD103
:102DD000AA7805A93B88087130000A704B80FEF77D
:102DE00047FBA0E7C843FF1F287A02111D4B37B5E8
:102DF000050098420BD000290AD1FFF777FF002881
:102E000005D11948FFF772FF002800D0058037BDB3
:102E100001291AD1FFF76AFF041EF8D001235B4293
:102E20000380A378FF2BF2D0FE2B07D00023E0789D
:102E30001422009329001E3300F022FBA01C00F096
:102E400044FB01235B426380E1E70229DFD10139C2
:102E500001F0AEF80028DAD12800FFF747FF041E82
:102E6000DFD1D4E7FEFF0000FFFF0000022210B513
:102E7000074B52421A80074801325A809A80DA8002
:102E800000F06EFA044801F015F8002010BDC046AD
:102E9000EC64FF1F112D0211ED2D02110388F7B50F
:102EA0000400002B02D102252800FEBD4268022149
:102EB000137825485268FEF7A5FD00282ED0234F31
:102EC00001253A88002AEFD0802321885B02012562
:102ED0009B1A9942E8DC0C2004F07AFA061E31D0E5
:102EE0003B8822889C4600231800019561469DB2CC
:102EF000491989B2AA421BD8002801D062443A80FD
:102F000000233000082208C0210004F031FB104AE1
:102F10001368002B13D100251660C5E762680221F3
:102F200013780C485268FEF76DFD0028C7D1BAE748
:102F300060681D014019418101330198D6E71A00EC
:102F40001B68E6E71325AFE7967A0211C643FF1F19
:102F5000E864FF1F947A0211014B18707047C04655
:102F6000C843FF1F14230A0010B51A40194204D0A9
:102F70000122102101F038F810BD4B06F9D40120D0
:102F800088434000F8E710B514008B0604D50122F1
:102F9000102101F029F810BD08230A001A40194237
:102FA00002D14BB2002B0FDA102101F01DF80028DE
:102FB00008D02300F9331B78002BECD0F8342378A9
:102FC000012BE8D10020E6E703208907FAD4E2E7E5
:102FD000F0B51F00184B85B01C6801900291039258
:102FE000002C27D1200005B0F0BDA5683301ED18F5
:102FF0006B89019A934211D3029A93420ED8002F03
:1030000004D10A9B002B10D12C00EBE73B00297860
:10301000039A6868FEF7F6FC0028F2D10136B6B2D2
:10302000A388B342E1D82468DAE7A3680A9A5B89E7
:103030001380E9E70026F3E7E864FF1F37B50C00CB
:103040000A8849880123914217D3002A15D0651DAB
:1030500023792A0002210A48FEF7D4FC1023002815
:103060000BD023796188208800242A000094FFF780
:10307000AFFF0A23A04200D0230018003EBDC04687
:10308000967A021113B50A000888498801238842FC
:103090000BD8002809D00024137905320094FFF7DB
:1030A00097FF0A23A04200D02300180016BD13B5D5
:1030B0000A0008884988012388420BD8002809D0D3
:1030C0000024137905320094FFF782FF0A23A042FF
:1030D00000D02300180016BDF0B58BB003904A88CD
:1030E00008880E000123824255D3002853D00023C4
:1030F000012704AC23700022718813000092FFF7AF
:1031000067FF051E3ED02078002835D12B78022B92
:1031100018D167706A8983000130E31880005A80F3
:1031200069680222201804F023FA23780133DBB205
:103130002370042B19D93B006889013080B2002B21
:10314000D9D01FE002236370122358436A892318E1
:1031500004305A8069681022201804F009FA237894
:103160000133DBB22370002BE5D10C4A6B899B182D
:103170005A425341DBB2DFE76378012BE4D12B786D
:10318000022BC7D022780A23002A04D021000398FA
:10319000FEF798F9002318000BB0F0BD0100FFFF07
:1031A0000F4BF0B504001868002816D083685D89BD
:1031B000A54207D88288AE18B44203DA12019A18E1
:1031C000934201D10068EFE71E005F891036A742E5
:1031D00004D1002900D00D801800F0BD3300EFE7C6
:1031E000E864FF1F70B505000C0008880021FFF798
:1031F000D7FF03000120002B04D022002800197AF9
:10320000FFF7C1FE70BDF7B50C000025019023004B
:10321000F6331B78AB4201D800200AE06B00E65A77
:1032200000213000E718FFF7BBFF002802D12680FD
:103230000130FEBD017A0198FFF794FE002802D00C
:103240003B882380F5E70135EDB2E0E710B50400D7
:1032500008880021FFF7A4FF03000120002B03D002
:103260002000197AFFF77EFE10BD0000054B1B6899
:10327000002B01D1180004E09A6852898242F6D1ED
:1032800098887047E864FF1FF0B50E27002687B0C6
:10329000039302ABFF183E8005001F4B40891400CA
:1032A000984207D02B78013000976A6880B2FFF708
:1032B0008FFE060002212B7818486A68FEF7A2FBF1
:1032C00000280FD06C892000FFF7D0FF002802D023
:1032D000013C0419A4B2039B002B00D01C803000D9
:1032E00007B0F0BD02212B780D486A68FEF78AFB13
:1032F0000028E7D102212B780A486A68FEF782FB92
:10330000002807D0002EDED03B88A342DBD1748991
:10331000013CDFE76C89DEE7FFFF0000967A0211CF
:10332000947A0211927A021170B504000D00160011
:10333000FFF7DCFC002803D083781720FE2B05D094
:10334000002E04D129002000FEF738F970BD0122BB
:103350001021200000F048FE0028F3D0F6E700001E
:10336000014B18607047C046F864FF1F37B56B46C5
:103370009D1D010004000222280004F031F92B8871
:10338000B02B0ED12379122B09D12300FF339B7868
:10339000012B06D10121608800F0E0F801E01B2B31
:1033A000F8D037BD10B5054B0421187000F098F81F
:1033B000FFF75CFDFEF780FB10BDC046FC64FF1FFD
:1033C0000020F0B50BB20F0087B0834234DA274BF0
:1033D000187804F0F5F9051E2BD00378A02B25D121
:1033E00003AE3100FEF7F4F8041E0BD1B378DB070F
:1033F00024D51F4B06341B68002B03D0310068888E
:1034000098470400A868002801D004F0C1F8002CF7
:1034100008D1184A039B1340174A934206D0B37849
:103420001B2B03D00121688800F098F8280003F0D6
:10343000D7FF80200002784007B0F0BD0F4B1B681B
:10344000002B10D0310068889847041EDAD07378BA
:10345000002BD7D1B27801A90A704B800C71688813
:10346000FEF706F8CEE70624F1E7C046FC64FF1F2E
:10347000F464FF1F00FFFF0000011200F864FF1F4B
:10348000F7B50190822040000D0017001E0004F0E7
:1034900057F904001320002C12D0B0232000237011
:1034A000089BFC226770658026710830002B08D0CD
:1034B000190004F05DF82100019804F099F900204A
:1034C000FEBD089903F0DCFFF5E710B5041E06D039
:1034D0000078FD2803D804F093F8FF23237010BD73
:1034E0000A1F93B210B504000220032B05D88240B6
:1034F0000020024BD1529B189C7010BD1C65FF1F11
:103500000B8870B5043B04000D000220032B0BD880
:103510000121200000F04CFD03001420002B03D0FB
:103520002900200000F0DEFB70BD000007B513008D
:10353000034A00920A00012100F02CFC0EBDC04697
:103540006937021107B5019203220092024B0A006B
:10355000122100F049FC0EBDE737021107B56B469A
:1035600001AA11800449D88008780633012802D1C5
:10357000190004F04DF807BDFD64FF1F0C4B10B59A
:1035800018700023FF210B4A1380138193819380CD
:10359000094A53801370517293819372D174D3820C
:1035A0001375517704F0BCF800F0FCF910BDC0466B
:1035B0002C65FF1F1C65FF1FFE64FF1FF0B58DB05B
:1035C0006B46002003910C229B5E834200DBB0E03F
:1035D0005D4B187804F0F4F8051E00D1A4E00378E0
:1035E000902B00D09DE006AF01004688380000F027
:1035F00013FA79680400002900D19CE03B88052B70
:103600006ED13B89032B1CD905AC200000F0A2F839
:103610006288172A61D83989131D994231D1796896
:10362000237804310291D90738D5607800F08EF9FB
:10363000071E06D0002303712378012B08D0132B1B
:1036400023D0A868002800D178E003F0A1FF75E03E
:103650006288029909A800F0A6F80290380000F0EC
:103660008BF909AA2378387A01920022310000925E
:10367000029A00F012F9380000F064F9029B002B66
:10368000DFD0300000F080F9DBE70378032BD8D1DE
:103690006288029909A800F0D6F8DEE7122B13D150
:1036A000029909A800F0B5F8021EEAD127498B88D3
:1036B000002BC6D0887909A92378019161780091FF
:1036C000310000F0EAF8BCE7002302AA938330003F
:1036D000617809AAFFF72AFFB3E71D4B0993F6E7C4
:1036E000042B02D09A1F012AABD8184A043B9B0036
:1036F000995A0029A5D0D218907831003A0000F0EC
:10370000AEF800289DD13B88042B03D00121300066
:10371000FFF724FF012C04D1A868002801D003F092
:1037200037FF280003F05CFE8020039B000243402B
:1037300018000DB0F0BD012800D182E70121300052
:10374000FFF70CFFEDE7C0462C65FF1F1C65FF1F50
:10375000010017000B7803704B784370CB788A78A0
:103760001B021343438070470A88030002700A88D3
:10377000120A42700A88012A06D14A8882704A8851
:10378000120AC2700420704702208242FBD14A888C
:1037900004309A704A88120ADA708A881A718A8804
:1037A000120A5A71EFE710B50400012082420CD9C9
:1037B0004B780A781B0213432380834206D1CB78CF
:1037C0008A781B0213436380002010BD022BFBD1BB
:1037D000CB788A781B02134363804B790A791B02EA
:1037E0001343A380F0E70B8803700B881B0A437018
:1037F0004B8883704B881B0AC3708B8803718B883E
:103800001B0A4371CB888371CB881B0AC3710820C4
:10381000704703000120082A14D14A780878120260
:1038200002431A80CA788878120202435A804A7981
:103830000879120202439A80CA79887912020243F7
:103840000020DA80704710B504000120022A05D15B
:1038500000204B780A781B021343238010BDF8B573
:10386000060010200F00150003F06AFF040001207D
:10387000002C0ED0A0230C22290023806780201D5D
:10388000002D07D003F074FE2100300003F0B0FFDC
:103890000020F8BD03F0F4FDF6E7F7B51E00009038
:1038A00008AB142017001D78019103F049FF041E96
:1038B00012D0A2230370019B47704380099B0571BE
:1038C00046710C220830002B07D0190003F050FE7F
:1038D0002100009803F08CFFF7BD099903F0D0FD9B
:1038E000F6E737B5041E0FD04388002B0CD0002517
:1038F000C1881323007A172201950095FFF7CDFFA9
:10390000FF2365806372257037BD000010B50C4938
:1039100004004A88002A09D08B89002B05D000209A
:10392000CB8A0222834201D010BD012213000A205B
:10393000434300204032C854C81842800472F3E761
:10394000FE64FF1F0023438003707047094B002172
:103950001A0010B55C88002C06D01C79844203D173
:103960000A234B43D01810BD01310A330329F1D18A
:103970000020F8E7FE64FF1F10B50400407A03F052
:103980003FFEFF23637210BD7047043010B580B254
:1039900003F0A6FE002803D00421494203F058FF9B
:1039A00010BD000070B50025104CA0682580A581D1
:1039B000A580A84202D003F0EBFDA56000250C4CC9
:1039C0000C4B606D1D80230058331D70A84202D03F
:1039D00003F0DEFD656500256068002801D003F076
:1039E000D7FD013508340A2DF6D170BDC465FF1F1F
:1039F0006865FF1FB865FF1F70B5041E09D1054D2E
:103A00002880A881A880A868002802D003F0C0FD03
:103A1000AC6070BDC465FF1FF0B54B8885B00193E5
:103A2000002343600A7905000F00022A00D07BE0E2
:103A3000CA88032A17D98B685E7819783602DC7831
:103A4000D8790E4399781B7A24021B020C43034356
:103A500053495BBA0B80331D93421ED1042C04D012
:103A6000631F022B0ED9012015E0019A4D4B120164
:103A7000D35A002B06D00198FFF7BEFF4A4A1369BC
:103A8000013313610421B8682E812C80494203F070
:103A9000DFFE6860002005B0F0BD434D042C06D069
:103AA000631F022B0FD9EB680133EB60DBE7019A50
:103AB0003C4B1201D35A002B05D00198FFF79CFF15
:103AC0002B6901332B61374B30000293019B029A23
:103AD0001B010193002301998C468B521300634410
:103AE0009C8003939E81FFF750FF039B041E986008
:103AF00016D00421B868494203F0AAFEFA880100F2
:103B0000043A200003F034FD0199029AFB888A5A96
:103B1000043B9B18029A8B522B6801332B60A2E75F
:103B2000AB690133AB619EE71E4B0293019B1E0103
:103B3000029BF35A002B2DD002998C19A068002803
:103B400028D0012A26D1FA889B189BB27352A189EA
:103B5000994217D39B1AC018B96803F009FD029B5C
:103B6000A289F35A934200D07DE700222B81A388DB
:103B70002B80A3686B60029BF2520B4A536801339F
:103B8000536070E7084A9368013393600198FFF728
:103B900033FF68E7044A536901335361F6E7C046CF
:103BA0002E65FF1FC465FF1F3465FF1F70B5051E1E
:103BB00015D10B4C0B4B1880230058331870606DD7
:103BC000002802D003F0E4FC6565250050356068EC
:103BD000002801D003F0DCFC0834AC42F7D170BD02
:103BE0006865FF1FB865FF1FF0B51700A12285B0FB
:103BF000920001934243394B06001B680C009B184E
:103C0000D933FF331D78FDF751FF0430854204DDC1
:103C10003000FDF74BFF0430C5B2BD4207D33A0078
:103C200000213000019B03F0ABFC05B0F0BD290082
:103C3000380003F09DFD2300C6B250331E7003937D
:103C4000019B29006365380003F03AFDCBB2029373
:103C5000002B02D0039B01361E7000262300503338
:103C600003931B78B34204D8606D002831D1002043
:103C7000DBE7029A2800002A04D0013B1000B3427F
:103C800000D02800F700E719387003F059FC78607D
:103C900000280ED03A78019903F06AFC019A3B782B
:103CA0000136D3180E4A0193D369F6B20133D361BA
:103CB000D4E7039B18706065A74205D1084A13201A
:103CC000D36A0133D362B0E7606803F061FC083463
:103CD000F2E703F05DFC00236365C8E73409FF1FCA
:103CE0003465FF1FF7B50D0007000421686803F075
:103CF000AFFD2B89040003702B891B0A43702B88AE
:103D000083702B881B0AC3702E8902250436F6B2F5
:103D1000FB2E15D81B4B9F4214D10C2003F010FD35
:103D20001135011E0CD0902303708E3B0371043BB0
:103D30004380154B8460C680187803F059FD002538
:103D40002800FEBD5C237B43104AD31800935833F0
:103D500001931B78002B0FD103003200380000992B
:103D6000FFF742FF019B05001B78002BE8D13800CC
:103D7000009903F025FCE3E7054A0725536A013360
:103D80005362DDE7FEFF00002C65FF1F6865FF1F23
:103D90003465FF1FF0B587B0009017200F001600A4
:103DA0000193FFF7F2FD1325041E19D00C98031E92
:103DB00002D00199201D9847030AE370052302AA47
:103DC000A0700430908127700098667003A99380DA
:103DD0000494FFF787FF051E02D0200003F0D8FBF4
:103DE000280007B0F0BD0000F0B587B01F000CAB95
:103DF0001B780391059301210DAB06001C780492FA
:103E000000F0D6F81425002821D02000FFF77EFD11
:103E10000135041E1BD01149059B0A78037001323D
:103E2000D2B2131EC68001D101231A000B70227179
:103E30003000049B03990097FFF7ACFF051E09D1E2
:103E4000230021000648074A093303F089FB2800B4
:103E500007B0F0BD002363802370F8E73065FF1FD3
:103E6000E338021130750000F8B505000E00064C6D
:103E7000064F2368002B02D03100280098470434F5
:103E8000BC42F6D1F8BDC046D465FF1FE865FF1FF0
:103E90000123064A5B425380002313715362044A94
:103EA000136053609360D36013617047E865FF1F30
:103EB000D465FF1F0200002310B506499C00085975
:103EC000002801D1625010BD0133052BF6D113201B
:103ED000F9E7C046D465FF1F034A5388181A4342C6
:103EE0005841404210407047E865FF1FF0B585B06B
:103EF00002930AAB1F780CAB1B88009008000E00E1
:103F000001920393FFF7E8FF05001120002D1BD15C
:103F10000E48FFF7E1FF04001520002C14D0062204
:103F20000B99A771E01D03F023FB019B3000237167
:103F3000029B29006371009B66802370039B65626E
:103F4000E381FFF791FF280005B0F0BDFFFF0000FF
:103F500010B5FFF7C1FF04000220002C12D06088CA
:103F60000121FFF781FF606A002801D003F080FB88
:103F700028220021200003F083FA012300205B4265
:103F80006380207110BD000030B5074A074C55888A
:103F9000010013780020A54204D05B1A59424B411E
:103FA0005842104030BDC046E865FF1FFFFF0000CB
:103FB000084A10B501230C00904208D0FFF78CFF8F
:103FC000031E04D0037923405A1E9341DBB218002C
:103FD00010BDC046FEFF0000024B1879431E9841F9
:103FE000C0B27047E865FF1F70B504000D001600F1
:103FF000FFF772FF002804D10D4B9C4200D0143013
:1040000070BD416A03790520002907D012221A40A9
:10401000102A02D10520002EF2D10F20DB06EFD5A9
:10402000897E0C20A9428941494249420840E7E77C
:10403000FEFF0000030010B5002800D110BD0348AA
:10404000034A41889142F9D09847F7E7E865FF1F96
:10405000FFFF0000002330B5C45CCD5C6C40D4543D
:104060000133102BF8D130BD0F23002210B5C45CF2
:1040700064002243CA54C25CD209013BF7D210BD8E
:104080000200010010B52032103103F089FA10BD92
:10409000F0B58BB00390102005931700049103F046
:1040A00097F90090102003F093F9009B13240190DE
:1040B000002B05D000280CD11324009803F0D8FA67
:1040C000019B002B02D0180003F0D2FA20000BB0A5
:1040D000F0BD102003F07CF90600102003F078F901
:1040E00013240500002E00D1AEE0002819D01022C4
:1040F000002103F0C5F932002900039803F050FABB
:10410000041E0ED133787F2B51D830000099FFF771
:10411000ABFF009B1B787F2B53D801990098FFF7CA
:10412000A3FF300003F0A4FA002D02D0280003F012
:104130009FFA002CC1D1102003F04AF9060010208C
:1041400003F046F90290002E7CD0002878D03A0087
:104150000F3223000125121105D00F333B4015B259
:104160005A4253411BB26A1E1201002B33D0049BEA
:10417000D2B298180099029AFFF76CFF013D102205
:104180000021300003F07CF9ADB2049F2D017D19B0
:10419000AF4242D0002C33D0300003F069FA029BCA
:1041A000002B00D189E7180003F062FA85E72900A7
:1041B0003000FFF759FF28002549009AFFF74AFF12
:1041C000A7E729000098FFF74FFF28002049019A30
:1041D000FFF740FFA5E70F210F4004998A18D9B2D5
:1041E0008F4208D9D15C06A819540133102BF6D19F
:1041F000029A0199C0E7791A48424141C901F2E7A0
:104200003900300006AAFFF725FF3200039806A9FF
:1042100003F0C6F910370400BAE7002CBCD1300017
:10422000029906AAFFF716FF320006A9039803F0C9
:10423000B7F9082204003100059803F099F9ABE7BB
:104240001324A9E71324AAE7002800D06EE733E778
:104250009C7A0211F0B58BB00F0016000225009079
:1042600000283FD0002A3DD00B1DDBB2180002937E
:1042700003F0AEF81135041E34D0FDF757FD0500EC
:104280003A000099201D03F053F8EBB20393E3705A
:104290002B0CDBB22F0A00936370FFB22B0E23703E
:1042A000A7700193FDF73CFD1022010006A803F062
:1042B0003FF82100029A04AB06A8FFF7E9FE051EAD
:1042C0000DD1039B08223370009B04A9B370019B9E
:1042D0007770F370301D03F02BF8FDF72DFD2000F3
:1042E00003F0C6F928000BB0F0BDF0B58FB00D009B
:1042F000149E039004920593002A03D10224200007
:104300000FB0F0BD002EF9D00398FFF7E5FD14249F
:10431000071EF4D07278337812021A43B3781B0464
:104320001343F27812061A43036A0192934201D3AF
:104330000133E3D1002D03D03B7901249B07DED567
:104340000822002106A803F09BF8059B13240433E0
:10435000DBB21800029303F03BF8051ECFD0059A9C
:104360000499043002F0E4FF04223100280002F036
:10437000DFFF3900102210310AA802F0D9FF29000E
:10438000029A06AB0AA8FFF783FE041E0FD108228B
:1043900006A908A802F0CCFF0822311D08A803F0E6
:1043A00077F8012807D101990398FDF7D9FC280077
:1043B00003F05EF9A3E70124F9E7000070B51C4C97
:1043C00005002368181E10D0002D14D11A78002A79
:1043D0000CD1981C083203F0CBF802F0D1FF013564
:1043E000002808D123681D70012070BD0A33180011
:1043F000082203F0BDF82368002BF5D0122003F04B
:104400009FF9061E0DD0C12321680370457002314B
:104410001022023003F0ACF823683100587803F022
:10442000E7F9206803F024F900232360DCE7C046A5
:104430001066FF1FF8B504002020FDF765FB0D4E48
:10444000A700BB590500002B0DD000280BD0D87851
:10445000FF2809D108492A000C55F35907480333AE
:10446000611803F07DF8F8BD290003F0C1F80028B9
:10447000F0D1F8E72C66FF1F1466FF1F8D5602115E
:1044800070B5064D84006359002B05D0D87803F031
:10449000B7F8FF226359DA7070BDC0462C66FF1F63
:1044A00070B506008CB00C00150000213022684663
:1044B00002F0E6FF31001022684602F039FF1D20AD
:1044C00021000322684402F033FF6846FFF7D8FD5D
:1044D0002D21040003222800694402F029FF200056
:1044E0000CB070BDF0B50700160097B001931CAB7F
:1044F0001D7830221EAB00910AA800211C7802F022
:10450000BFFF102239000AA802F012FF102200217A
:1045100002A802F0B5FF0722310002A802F008FF4E
:10452000072202AB9818631E9C41019902F000FF1C
:1045300002AB9C732B005A1E934102AAD373002135
:10454000102206A802F09CFF06221D9907A802F07F
:10455000EFFE1A2002ABC01806221F9902F0E8FEF7
:10456000102200990EA802F0E3FE102202AB0EA961
:1045700008781C78013A6040D2B2087001330131EA
:10458000002AF5D10AA8FFF77BFD102212A904002A
:104590000EA802F0EDFF102206AB0EA908781D78D8
:1045A000013A6840D2B2087001330131002AF5D1D6
:1045B0000AA8FFF765FD044310222098E4B212A96F
:1045C00002F0B6FE200017B0F0BD70B50E0014006A
:1045D0008CB00100102268461D0002F0A9FE3100D7
:1045E000082204A802F0A4FE2100082206A802F076
:1045F0009FFE6846FFF744FD04001022280008A92A
:1046000002F096FE20000CB070BDF8B506000D005B
:1046100000243719AC4200D3F8BD02F059FF030A59
:104620003B70631CDBB201379D4203D90234F05466
:10463000E4B2EEE71C00EDE773B506000C000225BE
:10464000002819D0002917D0032101A8FFF7DDFFAA
:104650006B469A793F231A40013313436A46300070
:10466000937101A92200FFF71BFF051E04D103224D
:10467000E01C01A902F07CFF280076BD03785807F2
:10468000DA08C00FD20080009B0710439B0F18432D
:10469000C0B2704707230B40C908C9000B43037021
:1046A0007047000070B50400FFF7EAFE134DA40048
:1046B0006359002B21D0186A002801D002F0D8FFDE
:1046C0002B59986E002801D002F0D2FF2B59D86EDA
:1046D000002801D002F0CCFF2B59186F002801D020
:1046E00002F0C6FF2B59586F002801D002F0C0FF1E
:1046F000285902F0BDFF00232B5170BD2C66FF1F0F
:104700000E4B8000C35870B50C00002B0FD09D6875
:10471000002D0CD02B78201D0B706B784B70A97C72
:10472000FFF7B8FF2B7E23726B69E36070BD102228
:104730000021200002F0A4FEF8E7C0462C66FF1F0F
:10474000014B18607047C0462866FF1F074A0300E8
:104750008000825810B5002A06D0D088984203D134
:10476000012901D1FFF79EFF10BDC0462C66FF1F37
:10477000F0B5264E95B087000B93BB590500099103
:1047800012200A92002B31D0D888FFF7A5FB040035
:104790001420002C2AD0280010A9FFF7B1FFBB5924
:1047A0001E781D6A002E23D00895FDF7FFFA07003A
:1047B0000020FDF701FB0790A379E61D069310ADDD
:1047C0000CA9089800F0E2FA0EA9280000F0D7FA28
:1047D0000B9B0A990493069B09980293079B0396E7
:1047E000019300970EAB0CAAFFF77CFE15B0F0BD4D
:1047F000FDF7DCFA06903000FDF7DEFAE31DA7793D
:10480000079310AB06000893DAE7C0462C66FF1F3B
:1048100030B50C4C85002A59030085B00120002AD0
:104820000ED018006946FFF76BFF2B591A78D8880D
:10483000054B002A00D1054B6A46072100F0D9FB41
:1048400005B030BD2C66FF1F7F4D02118D4D02114A
:1048500030B5094C8500295985B0102268462531AC
:1048600002F086FE2A591121044BD0886A4600F0D6
:10487000C0FB05B030BDC0462C66FF1F294E02119B
:1048800030B5094C8500295985B01022684635316C
:1048900002F06EFE2A591121044BD0886A4600F0BE
:1048A000A8FB05B030BDC0462C66FF1F674E021145
:1048B000F7B54D4F86001020F4590D0002F088FD29
:1048C000F3592062186A132200286CD0033A290099
:1048D0009C6802F04DFEF3591A780192002A58D1D3
:1048E0001E6A227D317B944651400122019F114274
:1048F00001D167461740217D914339432175377BAC
:104900004F40BC4660460027800701D44F0817403F
:10491000012102208F40227D82433A432275377B5A
:104920005740BC4660460027400701D497080F4017
:104930000420227DBF0082433A432275627D002716
:1049400094466046727B42400A4201D167460F405E
:104950000121627D8A433A436275777B5740BC46AA
:1049600060460027800701D457080F400220627D6F
:104970007F00824317436775767B00227E4076076F
:1049800001D4BA080A400426617D9200B1430A436B
:1049900062756A78002A08D06278002A05D005225C
:1049A0000533DA7700221000FEBD04222979114276
:1049B00005D1A17C114202D10533033AF1E7019AF6
:1049C00021782C78002A02D10A0021001400182234
:1049D0000429E8D8042CE6D805206043034A0533AF
:1049E0001218525CDDE7C0462C66FF1FAC7A02113C
:1049F00010B50A001121024B00F0FBFA10BDC046B1
:104A0000C34E02110B0030B587B001AD2B806B4651
:104A100004001100981D082202F0AAFD2A000B21B3
:104A20002000024B00F0E5FA07B030BDEB4E02115A
:104A300010B50A001121024B00F0DBFA10BDC04690
:104A40003F4F021113B50B0011006A4613706B46FD
:104A500004000622581C02F08BFD6A460821200043
:104A6000014B00F0C6FA13BD5F4F021110B50A00EA
:104A70001121024B00F0BDFA10BDC046AF4F02112C
:104A80007FB505000B4BAA00D4580800002C0FD0AE
:104A9000666F237FE28821780396266F0296E66E82
:104AA0000196A46E0094FDF719FC2800FFF7FAFDAB
:104AB0007FBDC0462C66FF1F10B51721FFF7E0FF32
:104AC00010BD000070B50A000D00064B0221040065
:104AD00000F08FFA060029782000FFF7D1FF3000A0
:104AE00070BDC0468F4E021170B586B000236A4675
:104AF0001370836804001D78681E0A2859D801A91C
:104B000002F07EFC060633373B3F43474B4F5300D2
:104B1000180000F042F9062312284BD000281BD1C0
:104B20006088FFF7D9F90823002813D04279002ABA
:104B300047D1264B1A78072312070BD5244B1A6846
:104B40000723002A06D01668002E03D0290001AAE8
:104B5000B04703006A4613706B461B786088002BD1
:104B60002AD1FFF767FC06B070BD180000F06CF9A1
:104B7000D4E7180000F087F9D0E7180000F093F9A7
:104B8000CCE7180000F0ADF9C8E7180000F0C3F951
:104B9000C4E7180000F0F6F9C0E7180000F0F6F9D5
:104BA000BCE7180000F013FAB8E7180000F013FA99
:104BB000B4E707236A46137069466088FFF782FFEF
:104BC000D1E70523012AC5D1024BB8E7B964FF1F1D
:104BD0002466FF1F2866FF1FF8B52C4F8600F35987
:104BE00004000D00002B40D0DA8882423DD15A7873
:104BF000062A33D11A78002A2ED0012099681A6A21
:104C0000097D014206D0157B054203D007225A7068
:104C10000120F8BD0220014204D0157B054201D0DD
:104C20000922F4E70420014204D0127B024201D0A1
:104C30000B22ECE7164B1B68002BE9D05B68002BBE
:104C4000E6D020009847BB5900215B78122BDFD1BA
:104C50002000FFF715FFDBE70E4BECE7112A04D12C
:104C6000002900D032252900F2E7002D08D12000CC
:104C7000FFF732F9002803D01023027913430371A0
:104C800021002800FDF7A8FAC2E7C0462C66FF1FE6
:104C90002466FF1F2866FF1F70B50E4E8500AB59B6
:104CA0000400002B13D01B78002B11D10A4B1B687A
:104CB000002B04D05B68002B01D02000984773596B
:104CC0005B78122B03D100212000FFF7D9FE70BDC5
:104CD000024BECE72C66FF1F2866FF1F2466FF1FB0
:104CE000094B8000C3581020002B0CD01A6A002AF0
:104CF00009D09B68002B06D0127A1B7E101C9A42AA
:104D000000D9181CC0B270472C66FF1F70B5030095
:104D10000D0014000220002A30D000292ED013707C
:104D20000B78081D53704B789370FFF7A7FCE07069
:104D3000012002212B7A23716B7B034063716A7B14
:104D40000A401343042263716E7B16403343637140
:104D50006E7BF608F600334363712B7B0340A3712F
:104D6000287B014000200B43A371297B0A40134399
:104D7000A3712A7BD208D2001343A37170BD10B572
:104D80000A0001000120FFF7C1FF10BD10B50A00A5
:104D900001000220FFF7BAFF10BD70B506000C003D
:104DA0000220002E30D000292ED07378201D0B70E9
:104DB000B3784B70F178FFF76DFC012235792572DD
:104DC00071794B1008001340934010400343881042
:104DD00010408000C9080343C9000B436373B179D5
:104DE0004B100800134093401040034388100240CA
:104DF0009200C9081343C9000B4321202373FCF719
:104E000083FE854201D2122070BD2220257AFCF754
:104E10007BFE8542F7D823781820042BF4D86378DA
:104E2000012BF1D80020EFE7030010B50220002984
:104E300009D0002B07D00322481C0A7019000D323C
:104E400002F096FB002010BD03000222080010B5FE
:104E5000002B06D0002904D00E32591C02F088FB2A
:104E60000022100010BD030010B50220002909D057
:104E7000002B07D00422481C0A7019000C3202F0E3
:104E800077FB002010BD10B5FFF7DEFF10BD03005B
:104E90000220002906D0002B04D0052200200A7031
:104EA0001B784B70704703000220002B08D00029AC
:104EB00006D05B7800200B70013B082B00D918301E
:104EC0007047030010B50220002909D0002B07D03D
:104ED0000622481C0A7019000A3202F049FB002021
:104EE00010BD10B5FFF7B0FF10BD02000B0002208F
:104EF00010B500290ED0002A0CD007211970118896
:104F000059701188090A997011180822D81C02F0EA
:104F10002FFB002010BD03000A00022010B5002B5B
:104F20000CD000290AD099785878090201431180E1
:104F3000901CD91C082202F01BFB002010BD0300AE
:104F400010B50220002909D0002B07D00822481CE8
:104F50000A701900921802F00BFB002010BD02002D
:104F60000B00022010B500290BD0002A09D009211E
:104F70001970117818185970511C062202F0F8FAAD
:104F8000002010BD10B5FFF75FFF10BD02000B0041
:104F9000022010B5002A09D0002907D051781970D5
:104FA00011180622581C02F0E3FA002010BD03007D
:104FB00010B50220002909D0002B07D00A22481C76
:104FC0000A701900063202F0D3FA002010BD10B5A5
:104FD000FFF73AFF10BD02000B00022010B5002AB7
:104FE00006D0002904D018005178FFF753FB0020A9
:104FF00010BDF0B585B017001E006A4606230500F7
:10500000080091819380FEF7C0FC1324011E0290DA
:105010000CD03800B047041E05D1280001A9FEF7C6
:105020006FFA041E02D0029802F0B2FA2800FFF7CD
:1050300001FA200005B0F0BDF0B504008BB001917D
:1050400015000021102202A802F01AFA334EA70020
:10505000B85900283CD0C388A34239D10378002B2B
:1050600036D14278062A18D1020001005532353176
:105070000C3006ABFFF7A9FA002829D12000FFF772
:105080002FFE020006A902A802F072FA200002A96F
:1050900002F056F901200BB0F0BD816E002917D047
:1050A0000B8A112A28D19D420ED101981231093A5A
:1050B00002F0EEF9012807D1BB5920009D6EFFF7E1
:1050C0000FFE29000200DEE732212000FFF7D8FCA6
:1050D0002000FEF701FF061E1BD0416A002918D0F0
:1050E0000B8AAB4215D108220198123102F0D0F997
:1050F00001280ED1716A0AE09D42E9D10822019887
:10510000123102F0C5F90128E2D1BB59996E8A7EAD
:10511000B9E7200002F0FCF8BCE7C0462C66FF1F90
:10512000F0B56B4D87007E5985B0337802900393BC
:10513000002B00D087E0B368346A019370780628AA
:1051400017D101221B7D134202D0217B114218D1BD
:105150000222134202D0217B114251D10422134278
:1051600003D0237B134200D08BE0019B5A7DEB5987
:1051700091E007380428F8D802F042F9032E42677C
:105180008300B36E002B03D11C2002F021F9B0661E
:10519000EB599C6E002C1CD010220021200002F044
:1051A0006FF90298FFF79CFD01002000FFF72DFA30
:1051B00002F08EF92082200008211230FFF725FA34
:1051C0000298FFF78DFDA076EB592100D888FFF7F4
:1051D0000FFC0822EB591CE0B36E002B05D01A001F
:1051E000198AF0881232FFF70DFC0222019B197D0B
:1051F000EB5911423DD0207B10423AD0073208E0F3
:10520000F488FCF7EBFD01002000FFF711FC0A22F7
:10521000EB595A70029B9C002A595378073B042B88
:1052200011D8D088FEF758FE00284ED0C3895A08FE
:10523000D2182849029B0298CB542B5941180433A9
:10524000254802F08DF905B0F0BDFCF7AFFD030075
:105250000120834201D100200393EB59DE88FCF743
:10526000ABFD039902003000FFF7ECFB019AEB590C
:10527000117D042211420CD0217B114209D00B2256
:10528000C7E7F688FCF74CFD01003000FFF7EEFBA6
:105290006BE7019A527D01210A4204D0607B0842EB
:1052A00001D00C22B5E702210A4204D0607B0842FB
:1052B00001D00E22ADE704210A4204D0627B0A42EB
:1052C00001D01022A5E71222A3E7FA225200B0E78C
:1052D0002C66FF1F3066FF1F9756021110B5064B54
:1052E0001A780423100018401A4200D00348FFF730
:1052F00027FA002010BDC046B964FF1FCC43FF1F32
:1053000070B50400FFF7D4FA051E43D12000FFF763
:105310007FFA234EA400A0598268937CDB0708D54E
:105320000321036A1B790B40012B02D1017F0B4340
:105330000377431DD97F8B1E022B0DD8022900D085
:105340000121C088FCF7A0FF042133591A7F59704E
:105350000A431A77280070BD01290CD102231022BC
:10536000437000210C3002F08BF830591021353099
:10537000FFF74BF9EEE70529ECD10223D118437072
:1053800010220C3002F0F4F804233259117F0B4341
:105390001377EAE708251828DCD1053DDAE7C0468F
:1053A0002C66FF1FF0B58BB0059143887E4F9E00A1
:1053B000F45915000493002C15D1012902D00020C6
:1053C0000BB0F0BD101D57781678FFF757F9EB6852
:1053D000320002932B7A0499019300903B00200045
:1053E000FCF71CFFEBE7E388049A934201D0082006
:1053F000E6E72378012B00D1D4E0059B581E09284D
:1054000000D9CFE001F0FCFF05CE0A29CC506C8515
:105410009AB229000498FFF773FFD1E72000290012
:105420001022453002F0A4F8B9594B78042B02D170
:10543000013B4B70C3E70B000A00253335320C31BA
:105440000498FFF795F90498FFF702FA0522431E26
:105450009841BB59C0005A70B2E7200029001022C1
:10546000553002F085F8049B4F4C9D002959049853
:105470000A0006AB55320C31FFF77AF92959102290
:10548000453106A802F004F8012808D10498FFF776
:10549000F7F90590002804D106222B595A70059877
:1054A0008EE708230593FAE763780C2B7AD1E36E35
:1054B000002B03D11C2001F08BFFE066BB59D86E96
:1054C00000286FD01022290002F052F8BB5904982E
:1054D000DC6EFFF705FC0D22A076BB595A706EE713
:1054E000E06E00285ED063780D2B5BD12B880822FC
:1054F0000382A91C123002F03BF8BB599A68517D17
:105500000222114226D0186A407B104222D00C326F
:10551000E4E763780E2B45D1236F002B03D11620CF
:1055200001F056FF2067BB59186F002803D01022E6
:10553000290002F01DF80F22BB59CFE763780F2B2B
:1055400030D1206F0622691C103002F011F8BB59CF
:105550009A68517D0422114203D0196A497B114295
:10556000D5D100210498FFF78BFA28E7636F002B51
:105570000DD0BB59586F0028F3D01022290001F03C
:10558000F7FF0122BB5952425B6F1A61E9E7142011
:1055900001F01EFFBB5960675B6F002BE9D126E766
:1055A0002978DFE707200BE72C66FF1F10B5064CB4
:1055B000207001F03DFF06212078FDF791FF0348A0
:1055C000FEF778FC10BDC0463F66FF1F4D47021135
:1055D00000200BB270B50D00834216DA264B187806
:1055E00002F0EEF8041E0DD00378922B0ED0A02B03
:1055F00037D0224B1878FF283AD0210002F0F8F873
:10560000002835D180200002684070BD43780E2B01
:105610000BD03E2BEDD18378052B12D0082BE8D18F
:1056200081798088FFF7D8FA08E0154B82889A4282
:10563000DFD183681878591CFEF7C0FE002817D107
:10564000D7E7104B1B785B0712D50F4B1B68002B5D
:105650000ED09B68002B0BD0C289811D8088984793
:10566000ECE7FFF741FAA068002801D001F090FFB5
:10567000200001F0B5FEC5E73F66FF1FC543FF1FD1
:1056800018200000B964FF1F2866FF1F10B50078BE
:10569000FFF712FA10BD10B50078FFF7FDFA10BD44
:1056A0000C234343084A10B59B185A68002A03D0BC
:1056B000012901D1904710BD9B68002BFBD0002928
:1056C000F9D19847F7E7C0465C66FF1F10B516286A
:1056D00013D801238340094A946B1C439463506B95
:1056E00098435063D46B20009843012901D12000D6
:1056F0001843D063116B0B43136310BD008000404F
:10570000F0B500240127154B85B0DA6B144E0392D7
:105710001A6C0192DA64019BE3403B4217D0039D6F
:10572000E5403D400295E5B202992800FFF7B8FF39
:10573000316A736A002908D03900002B01D0029920
:1057400079402800FFF7C2FF01E0002BF9D10134B6
:105750000C36172CDFD105B0F0BDC04600800040EC
:105760004066FF1F10B5012402002000162A08D849
:10577000054B5968D140214204D01868D04001231C
:10578000184010BD186DF9E700800040162807D8B2
:105790000122064B8240002903D0D9680A43DA600F
:1057A0007047D9689143D960FAE7C0460038004095
:1057B000162807D80122064B8240002903D0596CD5
:1057C0000A435A647047596C91435964FAE7C046DA
:1057D0000038004030B5162818D8032444430F4B36
:1057E000E25C1B199C785D7801232D1B0135AB40D1
:1057F000013BA340A140DB430C00122807D8084915
:1058000092005218116819402143116030BD054AB9
:1058100011680B4023431360F8E7C046F37A021186
:1058200008F0004014F00040C21F70B5D4B2062347
:10583000092C0BD80125084C9540002908D00021DF
:10584000FFF7C8FF23682B4323600023180070BDB7
:105850002368AB43F8E7C04600380040F0B516288F
:1058600026D8214B1B185B78022B21D103244443FB
:105870001E4A1F4EA35C1219947801221500854020
:10588000B76B013CE4B23D43A240B563194C12280A
:1058900015D89B0000290CD117495B1899680A4359
:1058A0009A600123205C154A834011680B43136002
:1058B000F0BD11495B18996891439960F1E70E4B6F
:1058C00000290DD159690A435A61225C1328E8D096
:1058D0000123203A93400A49086803430B60E7E735
:1058E000596991435961F0E74066FF1FF37A02114D
:1058F00000800040387B021100F00040A0F0004022
:10590000A4F00040F8B500241B4E1C4D1C4B1B5D41
:10591000012B1FD1184A9269E2401A420BD0012292
:10592000AA5693402200143AD2B2022A09D8154945
:105930004A6913434B6101340C360235172CE5D10B
:10594000F8BD0022AA560F499200521891680B43E5
:105950009360F0E7022BEED1E7B23800FFF702FFC9
:1059600001235840C1B23800FFF778FF3800FFF735
:10597000F9FE7077DFE7C0464066FF1FC57A021167
:105980004166FF1F00F00040012202388240054BB3
:10599000002903D059690A435A61704759699143F4
:1059A0005961FAE70038004070B504000D00052089
:1059B000162C1AD800212000FFF7E8FEA31E012BA9
:1059C00003D801212000FFF7DFFF00212000FFF7AF
:1059D0002BFF01220A49A2400A4B4868012D05D13C
:1059E00002431B194A605D70002070BD90434860FF
:1059F00002211C196170996991439961F4E7C046CD
:105A0000008000404066FF1F10B516280AD801220A
:105A1000074B8240002906D019680A431A60012109
:105A2000FFF7C2FF10BD196891431960F7E7C04640
:105A30000080004070B505000520162D17D80C23F6
:105A400000246B430A4A21009B181C70094B280054
:105A50005B195C70FFF7A8FF0123AB4020000649EB
:105A60000A681A430A6005490A689A430A6070BDC9
:105A70005C66FF1F4066FF1F34800040308000409E
:105A800070B504000E00FF2813D003250540FFF772
:105A9000D1FF084AA3089B009B183F22ED00AA40B3
:105AA000AE40196820009143314319600121FFF78E
:105AB0006DFE70BD18380040F8B505000520162DA4
:105AC00025D80C246C43124BE4186368002B03D1D7
:105AD000A3680D30002B1AD0022201270D4B0021A4
:105AE0005B195A7028002770FFF75EFF63681E1E5F
:105AF00008D0A3683E00002B04D02800FFF732FE38
:105B00004640F6B228003100FFF7E0FD0020F8BD66
:105B10005C66FF1F4066FF1FF7B5C420FF222B4BBA
:105B200080001958002491437F3A0A431A5080227A
:105B3000274F5202274E1A60274B1D5D002D21D0A2
:105B4000A31E012B03D80121E0B2FFF71DFF012D99
:105B500018D11F4B9B69E3402B4213D0E3B21800CE
:105B60000193FFF7FFFD01000198FFF74DFFE3B23E
:105B7000143B022B1DD801217156184A8D405369E0
:105B8000AB4353613B7F002B0DD0E5B22800FFF7FC
:105B900093FF2800FFF7E6FD7B7F0100834202D0E0
:105BA0002800FFF77DFD01340C370236172CC3D1D6
:105BB000F7BD012100237156F3568D40074A9B0023
:105BC0009B189A68AA439A60DCE7C04600E100E0AF
:105BD0004066FF1FC57A02114166FF1F00F00040BA
:105BE00010B504000520162C0CD801212000FFF769
:105BF000DBFE0123044A002011194B70A340916978
:105C00000B43936110BDC0464066FF1F70B5150081
:105C100004000E00FFF70EFF0C236343084A200028
:105C20009B189D605E60FFF747FF064B064A051E06
:105C3000136002D02000FFF7FDFE280070BDC046B3
:105C40005C66FF1F01570211C003FF1F70B5134DA3
:105C500007202C78002C1FD1982221005200280008
:105C600001F086FB0123C420FF222B700C4B800027
:105C70001C635C630B4B1C605C600B4B19589143BD
:105C80007F3A0A431A50802252021A600D20074AB6
:105C9000074901F0EDFD200070BDC0464066FF1FC2
:105CA00000800040A0F0004000E100E0195B02111C
:105CB00005590211030010B50620072B07D8044A26
:105CC000137001F06DFB0020024B034A136010BDFE
:105CD000F443FF1F151BFF1F5C03FF1F70B51D0062
:105CE00002240C2910D8094ACA40D2070CD5FBF768
:105CF00017FF041E08D1059A04992800FBF72CFF12
:105D0000FCF79AFDFFF7EAFA200070BD12100000C0
:105D100030B50D7802232C009C43184201D02B4350
:105D20001C0008252300AB43284201D02B0023434D
:105D300020241D00A543204201D01C4325002A2316
:105D40000D70184204D011781E3B0B43137030BD08
:105D50000028FCD10C2113788B43F7E7F8B51D0020
:105D600006AB1B88140007AA0E000B201778002B27
:105D700027D10A78022A49D14A685078117800025E
:105D8000244A08438018042840D801F039FB031244
:105D90001D1B2300F06801F08BFB021CC0B2B8424F
:105DA00000D93A1CD2B22000F1682A8001F0E0FB51
:105DB00006E00222F3681B882A8023701B0A6370A6
:105DC0000020F8BD0622EEE701232B80F3681B7844
:105DD0002370F5E7F368002B16D008222A801A8872
:105DE00022701A88120A62705A88A2705A88120A9F
:105DF000E2709A8822719A88120A6271DA88A27116
:105E0000DB881B0AE371DBE72B80D9E701202B80BD
:105E1000D7E7C04600D6FFFFF7B516000A781D0089
:105E200008AB1F880C000123022A18D14A68507859
:105E3000117800022B4A0843801803280FD801F07C
:105E4000DFFA02254439E06801F032FBC0B20723D3
:105E5000B84204D37B190193152B02DD0D231800E2
:105E6000FEBDE0682A003100C01901F081FB6B46DD
:105E700000209B88E268D0541B4B1B68834203D0F0
:105E80001B68834200D098470023E8E70B23002FCC
:105E9000E5D1022DE2D1737832781B021343E26818
:105EA0001380114B1B68002BEED01B68002BEBD02E
:105EB0000120E8E70B23002FD1D1062DCED12A00F7
:105EC0003100E06801F054FBDEE70B23002FC6D160
:105ED000012DC3D132787533012AC0D8E3681A7016
:105EE000D2E7C04600D6FFFF4C68FF1F70B50C001C
:105EF0001500072837D801F083FA041436361B360C
:105F0000242E182015290BD8184E162200213000F7
:105F100001F0B6FA22002900300001F029FB002030
:105F200070BD18200229FBD11288114B1A80F6E7A8
:105F300018200829F4D10A000E48290001F050FB6E
:105F4000EDE718200129EBD10B4B10780B49DA69EA
:105F5000FFF7DEFEE3E718200129E1D1064B1078B8
:105F60000749DA6BF4E70220DAE7C0463468FF1F1E
:105F70007244FF1F6844FF1FF843FF1F2044FF1FA8
:105F80004044FF1F030010B50020DB0704D50721A4
:105F9000024A034800F08CF810BDC046507B021145
:105FA000F843FF1F054A03001068002803D08288C9
:105FB0009A4201D1806870470068F6E7506AFF1F77
:105FC0000A88030008009A4204D08A8804309A4262
:105FD00000D0002070470000F8B5F82200230D4FD4
:105FE0000D4E7968050042433370994200D07B60C2
:105FF0000A4C0021200001F043FA00231A007C60C3
:10600000AB4202D100203370F8BD01332280DBB2F5
:10601000F834F5E7506BFF1F4C6BFF1F546AFF1FEE
:1060200073B56B4601900600684615001980FCF7B1
:1060300035FF041E11D1002D0FD07689002E11D00E
:106040000C2001F0C5F900280ED0084A046013683E
:1060500086808560002B02D11060200076BD1A007A
:106060001B68F7E70224F8E71324F6E7506AFF1FDE
:10607000012100220A4B10B549420A4C198099802F
:106080009A719A70084B2070012019805A60FFF7AE
:10609000A3FF2078FCF760FF0448FDF70BFF10BD5D
:1060A0005468FF1F586BFF1F506BFF1F5D6102118B
:1060B000022310B5002802D0FFF7B2FF030018003A
:1060C00010BD0000030010B50020DB0704D504213B
:1060D000024A0348FFF7A4FF10BDC046647B0211CB
:1060E0007844FF1FF0B50E2687B003930CAB1F88D2
:1060F00002ABF6180500080031000292FDF750F8D7
:1061000004000120002C0FD03088FFF74BFF030064
:106110000E20002B08D05E68002E05D0210028003C
:10612000039B029A0097B04707B0F0BD0A4B10B529
:10613000984207D10122002352420A808B708A8044
:106140008B7110BDFFF73CFF0028FAD001235B42A2
:10615000038000238370F4E7FFFF0000F8B505001B
:1061600001290AD1134E00243388F827AB4219D0F5
:1061700028001149FFF7DAFF06E0022904D10139AE
:10618000FDF716FF0028EDD0F8BD3B0063437268B1
:10619000D018D35A002B09D03A00002101F070F931
:1061A0000134E4B2054B1B78A342EED801235B42D5
:1061B0003380DDE7506BFF1F5468FF1F4C6BFF1FE0
:1061C00010B5FFF7FDFE03000020834200D0987851
:1061D00010BD0000F0B589B01C000EAB80CB039061
:1061E0001E8810AB1B78049202930B7A0D00DB061D
:1061F00016D42B780593022B24D00498FFF7D2FEF7
:10620000002812D003689C46002B0ED0029B22006F
:10621000019329003B00644603980096A04705E0DF
:106220000498FFF7BFFE002802D10E2009B0F0BD90
:106230008368002BF9D00A22290003989847002888
:10624000D7D0F3E76B6858781A786B4B000210438D
:106250009842D2D8043B984210D2684B984242D020
:1062600015D8674BC0180128C7D80B20002EDDD1E8
:10627000EB681A7859683A80200028E0614BC01812
:10628000032800D979E001F0BBF8846A789E5E4B60
:106290009842B2D10B20002EC8D101233B80EB687D
:1062A00031001B7823706889013080B2FCF778FFD9
:1062B0003A88031E0ED0017802328A183A80428949
:1062C00062704289120AA27059680278E01C01F0DB
:1062D0004FF906E004323A8031000422601C01F0DC
:1062E000CFF80020A2E70B20002E9FD1EB6807A972
:1062F0001E8804233B80330A300026706370FCF74D
:106300004FFF051E28D004AB9A890E2304A95B1801
:106310003E49C668FCF7B8FF00280BD12B783C48F3
:106320006A680599FBF76EFB002803D1012304AAD4
:106330005B42D3813278022A06D17168201D01F0B8
:1063400017F93B8802333B800E2304AA9B181B8855
:10635000A3701B0AE370C4E704ABDE81F4E70B20F3
:10636000002E00D062E7E9680398FFF729FF0223B7
:106370003B802070000A6070B3E70B20002E00D035
:1063800054E70222EB681B883A8023701B0A637073
:10639000A7E7E86801F08CF8C2B203000720B24218
:1063A00000D243E70DD00299DBB27118994202DBAB
:1063B000921BD3B20293029BE9681A003B808919B1
:1063C0005AE70023F6E70B20002E00D02EE7072225
:1063D000EB683A801A7822705A7862705A88A270F4
:1063E0005A88120AE2701A792271DA886271DB889F
:1063F0001B0AA37175E7C0460429000002280000AB
:1064000000D8FFFFFFD6FFFF03280000FFFF0000BA
:10641000947A0211F0B58DB06B46002008912022CD
:106420009B5E83423DDAA64B187801F0C9F9071E3E
:1064300032D00378B02B2CD10079023816281FD81F
:1064400000F03EFF17001E001E001E0031001E005F
:1064500096001E001D011E0052011E0073011E0049
:10646000CD011E0050021E001E001E008E021E00E6
:10647000E302944B94491B8878880B80FBF702F861
:106480003800FCF773FF914B1B68002B01D03800DC
:106490009847380000F0A4FF8020089B000243408A
:1064A00018000DB0F0BDF6220021874800F0E8FF8B
:1064B0000BAA3B7B7989388900923A000D32FCF7B0
:1064C00087FD0400804B1B78002C3FD146E0804BB9
:1064D000788805937F4B4100CB5A0BAE073BDBB26C
:1064E00032880293002301937B4B21000693009393
:1064F000059BFFF76FFE744D002810D1069B3A8A6A
:106500001B889A420BD138000599123000F0C0FF69
:10651000002804D02B7862899B00EB185A80162340
:1065200006A81B18328820007989FCF7ADFE2B786D
:1065300004009A00AA1851880029C3D00133DBB2A5
:106540002B70002807D006A9C98A9180634A128857
:106550009A42BCD802E0012149429180002B04D02C
:1065600059497888FAF7C2FF8AE73E890A2479E018
:1065700000253E89574B06937B88069A5B009B5A01
:10658000033B9D4202DB002DF0D05BE0162206A803
:1065900012183B7B798900923A0030000D32FCF7EB
:1065A00017FD0590002858D04689017A7888FCF7B5
:1065B000D9FC041E44D1464B78880793069B4100C2
:1065C000C95A454B0439C9B206AAD28A0693029128
:1065D000019400930599079BFFF7FCFD041E2FD142
:1065E000069B39491A88931C002D26D14B80798847
:1065F000384B4900CB5A5119033B8B4220DD059B98
:1066000031485B8941190B71A91C0135C9B2EDB242
:10661000059145191B0A2B71059B2D490433181848
:1066200000F0A6FF2C4B059A1B88D318DDB22C4B2B
:106630009E4205D00136B6B29CE749889942D6D031
:10664000002D0CD0204C2800618801F0F9F8207052
:1066500021007888FAF75AFF12E7059CF0E7002C32
:1066600000D183E77B78142B00D109E716493B79E9
:106670004E800B700C717888FAF7FAFE00E716244A
:1066800006ABE41821003889FCF78AFD011E00D111
:10669000B7E1788822880F4C45002C5B0A4D013CFD
:1066A000E4B2029400240F4B01940095FFF792FD91
:1066B000041E00D014E129007888FAF737FFDFE6DE
:1066C000586BFF1F6443FF1F5C68FF1F5068FF1F6C
:1066D0005669FF1F8C64FF1F4C6AFF1F6243FF1F38
:1066E000FFFF00005E68FF1F162406ABE4182100C0
:1066F0003889FCF755FD011E00D182E17888228897
:10670000AE4C45002C5BAE4D013CE4B202947C895A
:10671000AC4B01940095FFF75DFD041E00D0DFE057
:1067200029007888FAF70CFFAAE60025A44B1D8003
:106730003B00FE331B78A24A78880792AB4208D907
:106740009E4B12880693069943005B5A013B9A427E
:1067500003DB0799FAF7FEFE92E616246B00FB189E
:10676000059306ABE418059B21001889FCF718FD7A
:10677000011E03D1059B01241E8973E77888924B83
:106780002288069C099343001B5B904E013BDBB2C1
:106790000293002300960193099BFFF71BFD041E43
:1067A00002D0059B1E895DE77B88069A5B009B5A99
:1067B000079A108832881218934202DC1B1A013B98
:1067C00033807F4C023032880999001900F0D0FEE6
:1067D0002388328801359B182380EDB2A8E70BAAE5
:1067E0003B7B7989388900923A000D32FCF7F0FB47
:1067F00000250590059B002B04D10A24002D00D113
:106800006EE060E0059B7888197AFCF7ABFB01002D
:10681000041E63D1694C6C4B788806940993069BDF
:106820004400E45A694B063CE4B20BAE328807934D
:106830000294019100930599099BFFF7CBFC041E7C
:106840004CD1079B5E491B881A1D002D30D14A8010
:10685000059B5B4C5A8963191A716B1C9BB2E31838
:10686000120A1A71162306A832881B18798905980E
:10687000FCF70AFDFF21AA1C2E1D03350B00059015
:1068800092B2B6B2ADB2002803D006ABDB8AD9B261
:106890001B0AA218651911712B714C4D301D2A88E5
:1068A0004949201800F064FE2B88F618B5B2A1E71C
:1068B0004988914207D17A8806995200525AEB18BA
:1068C000053A9A42C4DC3E4C2800618800F050FF33
:1068D000207021007888FAF747FED1E5002DF2D12B
:1068E0003E89BFE6162606ABF61831003889FCF75C
:1068F00057FC3D000400FF3500282DD0037A9B068D
:106900000CD400227B893989788800923A000C32B5
:10691000FFF7E8FB041E10D03E8915E03088FFF732
:1069200041FB00281AD08368002B17D021001222C7
:1069300078889847041EE4D0EEE7AB78002B02D1AC
:106940007888FAF721FE0026AB78002B00D097E577
:10695000002C00D194E585E60124DDE70E24DBE779
:10696000162506ABED1829003889FCF719FC041E22
:1069700047D0037A9B0611D4154A7B881188994227
:1069800003D01448814207D11380134BF8261D7899
:106990000023D9B2A94221D30924A1E72888FFF70F
:1069A00001FB00282FD08368002B2CD0210012225D
:1069B00078889847041EDFD092E7C0468C64FF1F9A
:1069C0005C68FF1F5E68FF1F5669FF1F4C6AFF1F50
:1069D000506BFF1FFFFF00004C6BFF1F310059433E
:1069E000546801336018615A0029D2D13C00083440
:1069F0002100F82200F0BCFD21007888FAF7CCFDD8
:106A00003EE501246CE70E246AE71D4B1A887B885B
:106A10009A4231D07888FAF7C9FD31E5F823059814
:106A200051684343CD18C95A00291FD03B7A012B26
:106A30000BD16C88AB887888AA1D0094FFF752FBB5
:106A4000041E02D000233B722E88F8220021280069
:106A500000F016FD00232B80059B0133DBB205936C
:106A6000084B05991B78064A8B42D7D801235B4215
:106A70001380002CCED0F5E5002634000596EFE714
:106A8000506BFF1F4C6BFF1F70B504000E0015000C
:106A9000FFF796FA031E08D131000548FFF790FA78
:106AA00003001120002B02D01C8000209D7070BDBF
:106AB000FFFF0000F8B50B4F06003B780D001400F7
:106AC000FF2B0ED00A2000F03BFE011E09D0B1239F
:106AD0000380002346800371C5800481387800F06C
:106AE00087FEF8BDB944FF1FF7B50F0008A90600DF
:106AF000088809A90B240988002821D10234022B17
:106B00001ED1557813782D021D432B008B43019322
:106B10007334002B14D1FB68300019000093FFF789
:106B20004FFB019C85420BD02A0030000099FFF7F3
:106B3000ABFF041E04D12A0030007989FFF7BAFFA9
:106B40002000FEBDF0B50E7885B003900AA8058838
:106B50000120022E0DD14C682778647824023C4332
:106B6000054FBC4205D10398DBB201960095FFF7B3
:106B7000BBFF05B0F0BDC0460229000003681A053E
:106B800008D1054A1033127803601203934201D3EF
:106B90009B1A03607047C046746BFF1F70B50400FA
:106BA0000D00160000F09CFC030029209B0611D16B
:106BB000094B07381A68A2420CD8084B1B781B03F4
:106BC0009B18A34206D9A30704D132002900200054
:106BD00000F096FD70BDC046706BFF1F746BFF1F09
:106BE000064B10B51C68844207D8054B1B781B0365
:106BF0001B19984201D200F053FD10BD706BFF1FAE
:106C0000746BFF1FF0B501240F00002589B00090C0
:106C100002920194604B019A1B78934207D8009B23
:106C20002120002B68D0012B65D1252064E05B4E2C
:106C3000707C3179FE2C03D9FF3CA4B2FE2C52D8D3
:106C4000019B181800F01CFE009B002B00D1317432
:106C50000B0301260493002D36D0A619B6B2049B6F
:106C60003501ED184D4B0422186807A92818FFF7C5
:106C7000B7FF06AB9A1D009B012B3FD0022B5DD0C6
:106C800013789B079B0F022B03D0032B30D0002BD4
:106C900015D113780C2201241340042B0FD106AB1D
:106CA000DD880C212D09280000F0EAFD4B1E9941DA
:106CB00028000C000C2100F0C3FD2418A4B20136FA
:106CC000B6B20025FF2E0ED8012CC8D93319023ECA
:106CD00032199BB2FE2A02DC013B9EB2BFE70125BE
:106CE000023BFF3B9CB2019B0133DBB2019391E776
:106CF0002D052D0D3D60002009B0F0BD13789B07D8
:106D00009B0F022B04D0032B00D18EE7002BD6D192
:106D1000032206AB06331B781A40022A08D13A68D0
:106D200007A9098892B2914202D1029B1D60E2E755
:106D30000C2201241340042BC1D1B0E711788B073A
:106D40009B0F022BA5D0032BD5D0002BB7D10C2540
:106D50003B6829400393042919D1138829001C0991
:106D6000200000F08DFD4B1E994120000591290067
:106D700000F066FD059B1C18A4B26543039BEB184D
:106D80003B60029B029A1B680133136097E7039BE9
:106D900001240C33F4E7C046746BFF1F5C6BFF1FCC
:106DA0004A4BF0B51B684A4CFF212360494B002633
:106DB0001B789BB02371102309224748A17163718E
:106DC00000F05EFB4E22002106A800F059FB3500C2
:106DD0002179A94213D8A379FF2B3CD1002523792F
:106DE000EAB2013BAB4244DC6374102300226382AD
:106DF0003A4B227401321A7000201BB0F0BD20689B
:106E00002F031022381802A9FFF7EAFE2068029A21
:106E1000824214D16B46A288998991420FD12D4AA2
:106E20009B7B1278013A93424EDA5E1B721E9641AA
:106E300006AA02365355A3710135EDB2C8E73818DA
:106E400000F056FA1022FF2102A800F019FBFF22E1
:106E500006AB5A55F0E7012EC0D0172200206A4435
:106E6000C3B29942C8D9431CD55C002D0ED018007E
:106E7000F6E723682803A27121001022C018FFF74B
:106E80008DFE01350028AAD01F20B6E74018013832
:106E900000F0F6FC0122114B61741A7028002A00E0
:106EA00001A90195FFF7AEFE019B00280AD0212819
:106EB00006D0C0B221289FD000289DD02A209CE770
:106EC00080235B01638297E7202096E7706BFF1FAA
:106ED0005C6BFF1F746BFF1F636BFF1F596BFF1F02
:106EE0000E4B70B51B78181E16D080240C4B00205A
:106EF0005D8A6401A5420FD21979587C1B7C401829
:106F0000C01A013800F0BCFCFF230C201B014B43CE
:106F1000641BE3185843000970BDC046596BFF1F3E
:106F20005C6BFF1F07B50A0005490300097827209D
:106F3000002904D001A926380193FFF763FE0EBD96
:106F4000596BFF1FF0B585B0070016001D000191B9
:106F500000F0C6FA2924800625D1244B023C1B7878
:106F6000002B20D0019B053C002B1CD0002E1AD0FA
:106F7000380002A9FFF7D6FF041E35D11C4B0422AE
:106F80001868029B03A9C018FFF72AFE02AB9A1DDE
:106F9000002D02D013881B092B80158800272D098E
:106FA000AE421ED22624200005B0F0BD2E1C0C2DB2
:106FB00000D90C26029BB6B20093019B3200D9196E
:106FC0000B4BAD1B1868009BF71918180430FFF71E
:106FD00007FE009B02A81033ADB20293BFB2FFF7C9
:106FE000CDFD002DE2D1DEE72524DCE7596BFF1F44
:106FF0005C6BFF1F0023F0B585B00500029300F025
:107000006FFA2924800627D1264B023C1B78002BDF
:1070100022D0280002A9FFF785FF041E3DD1224B94
:1070200004221868029B03A9C018FFF7D9FD02AB20
:10703000DE880C213609300000F022FC4B1E9941FD
:1070400030000D000C2100F0FBFB2D18ABB2250029
:107050000193019B9D4202D1200005B0F0BD124F6B
:10706000029E38680422301803A9FFF7B9FD0321F6
:1070700002AB9A1D9B7938688B4313703018042239
:1070800003A9FFF78BFD002809D1103602A80135AE
:107090000296ADB2FFF772FDDBE72524DCE71F2483
:1070A000DAE7C046596BFF1F5C6BFF1FF0B58BB072
:1070B00005001700039100F013FA2924800676D109
:1070C000484B023C1B78002B71D0039B053C002BE6
:1070D0006DD07B1E444A9BB2934268D8FFF700FFF5
:1070E0000134874263D8280004A9FFF71BFF00285A
:1070F00057D002230C2205A93801034348880D808C
:10710000104003434B80974254D900233E00029322
:1071100004AB9A1D0C2E52D9BB1B591E8B410C205F
:10712000117801339B0081430B430C3E1370B6B2C0
:1071300001902E4D04226C8A2B6805A9E4182B7C43
:1071400006A81B03E418049400F012FA039B029AA9
:1071500007A89918019A00F00BFA019B20001A1D4C
:1071600006A9FFF71BFD041E39D1029A019B944624
:10717000802263449BB202936B8A520110339BB20C
:107180006B8293420AD1287C2979013000F078FB88
:107190006B7C994202D0102329746B82002EB7D1E8
:1071A00005E02800FFF726FF01240028A1D02000D9
:1071B0000BB0F0BD04AB99790A439A71A5E70C2393
:1071C000042011780B40043B8343DBB2002B02D137
:1071D0000C3399431170F3B201930026A9E71F24E1
:1071E000E5E7C046596BFF1FFE0F00005C6BFF1FF9
:1071F000094A03001278272010B5002A0BD11A057E
:107200002138002A07D1012905D9044A1170044AFE
:107210001360FFF7C5FD10BD596BFF1F746BFF1F97
:10722000706BFF1F10B504000C4800F0A9FA0C4861
:10723000A16B00F0A5FA0B48E16B00F0A1FA0A4837
:10724000216C00F09DFA094B0948196800F098FA82
:10725000084B1B68002B00D09847FEE7A879021165
:10726000BE790211CD790211DC79021104ED00E042
:10727000EB790211786BFF1F002307B501A801937A
:10728000FFF7D0FF044A0548002110B5121A00F09C
:10729000F7F8F8F7B5FEFEE77C6BFF1FBC44FF1F55
:1072A00001B40248844601BC604700BFD1A500007C
:1072B00001B40248844601BC604700BF713AFF1F19
:1072C00001B40248844601BC604700BF253CFF1F53
:1072D00001B40248844601BC604700BFC539FF1FA6
:1072E00001B40248844601BC604700BF5D1700003E
:1072F00001B40248844601BC604700BF9138FF1FBB
:1073000001B40248844601BC604700BF8935FF1FB5
:1073100001B40248844601BC604700BF091B00005D
:1073200001B40248844601BC604700BFFD3BFF1F1B
:1073300001B40248844601BC604700BF45510100CA
:1073400001B40248844601BC604700BF311B000005
:1073500001B40248844601BC604700BF35550000B7
:1073600001B40248844601BC604700BF21240000EC
:1073700001B40248844601BC604700BFB70E00005C
:1073800001B40248844601BC604700BFD91B00001D
:1073900001B40248844601BC604700BF8552010029
:1073A00001B40248844601BC604700BF151BFF1FA3
:1073B00001B40248844601BC604700BF4D1F000075
:1073C00001B40248844601BC604700BF7932FF1F08
:1073D00001B40248844601BC604700BF3D4B010038
:1073E00001B40248844601BC604700BF434D010020
:1073F00001B40248844601BC604700BF851F0000FD
:1074000001B40248844601BC604700BF113CFF1F25
:1074100001B40248844601BC604700BFC52100009A
:1074200001B40248844601BC604700BF9934FF1F85
:1074300001B40248844601BC604700BFC926000071
:1074400001B40248844601BC604700BF3D180000FB
:1074500001B40248844601BC604700BF21460100D8
:1074600001B40248844601BC604700BF1DBC000057
:1074700001B40248844601BC604700BFA54F01002B
:1074800001B40248844601BC604700BF154D0100AD
:1074900001B40248844601BC604700BFCD4C0100E6
:1074A00001B40248844601BC604700BFB14E0000F1
:1074B00001B40248844601BC604700BFDD520100B0
:1074C00001B40248844601BC604700BF8539FF1FF4
:1074D00001B40248844601BC604700BF2951010045
:1074E00001B40248844601BC604700BFD530FF1F8D
:1074F00001B40248844601BC604700BFEDA500000E
:1075000001B40248844601BC604700BF59520100E3
:1075100001B40248844601BC604700BF013BFF1F25
:1075200001B40248844601BC604700BFE1AC0000E2
:1075300001B40248844601BC604700BF291C00001A
:1075400001B40248844601BC604700BF017F0000CF
:1075500001B40248844601BC604700BFED4A010007
:1075600001B40248844601BC604700BFA94601003F
:1075700001B40248844601BC604700BFE94C0100E9
:1075800001B40248844601BC604700BF5118FF1F88
:1075900001B40248844601BC604700BFD9490100DC
:1075A00001B40248844601BC604700BFE5480000C2
:1075B00001B40248844601BC604700BFC94A0100CB
:1075C00001B40248844601BC604700BF7D18FF1F1C
:1075D00001B40248844601BC604700BF6930FF1F08
:1075E00001B40248844601BC604700BF810E000020
:1075F00001B40248844601BC604700BF5147010006
:1076000001B40248844601BC604700BF1147010035
:1076100001B40248844601BC604700BFE117000086
:1076200001B40248844601BC604700BFF933FF1F24
:1076300001B40248844601BC604700BF51250000E8
:1076400001B40248844601BC604700BF4D39FF1FAA
:1076500001B40248844601BC604700BF0D520100DE
:1076600001B40248844601BC604700BF8D1200008F
:1076700001B40248844601BC604700BF014C0100D0
:1076800001B40248844601BC604700BFB932FF1F05
:1076900001B40248844601BC604700BF053AFF1FA1
:1076A00001B40248844601BC604700BF0D37FF1F8C
:1076B00001B40248844601BC604700BF6132FF1F2D
:1076C00001B40248844601BC604700BF090E0000B7
:1076D00001B40248844601BC604700BFF94C010078
:1076E00001B40248844601BC604700BFE92800009D
:1076F00001B40248844601BC604700BF056A00002F
:1077000001B40248844601BC604700BFDD37FF1F5B
:1077100001B40248844601BC604700BF1D4B010014
:1077200001B40248844601BC604700BF79180000DC
:1077300001B40248844601BC604700BF8B5201007F
:1077400001B40248844601BC604700BF1D4D0100E2
:1077500001B40248844601BC604700BFC51D00005B
:1077600001B40248844601BC604700BFC9A90000BB
:1077700001B40248844601BC604700BF090E000006
:1077800001B40248844601BC604700BFE53A0100ED
:1077900001B40248844601BC604700BF4550000068
:1077A00001B40248844601BC604700BF75A90000CF
:1077B00001B40248844601BC604700BF691F000055
:1077C00001B40248844601BC604700BFF54E010089
:1077D00001B40248844601BC604700BF6DBC000094
:1077E00001B40248844601BC604700BFE936FF1F70
:1077F00001B40248844601BC604700BF594F0100F4
:1078000001B40248844601BC604700BF3934FF1F01
:1078100001B40248844601BC604700BF2526000031
:1078200001B40248844601BC604700BF9DA9000026
:1078300001B40248844601BC604700BF0124000037
:1078400001B40248844601BC604700BF350E000009
:1078500001B40248844601BC604700BF554901009D
:1078600001B40248844601BC604700BFB54C01002A
:1078700001B40248844601BC604700BF0133FF1FCA
:1078800001B40248844601BC604700BF350E0000C9
:1078900001B40248844601BC604700BF055E000099
:1078A00001B40248844601BC604700BFCD30FF1FD1
:1078B00001B40248844601BC604700BFB3520100D6
:1078C00001B40248844601BC604700BF5522000055
:1078D000000301030203030304020502060207007A
:1078E000080309030A030B030C000D000E030F032A
:1078F000100311001303140315031603B50302113B
:10790000E9030211000000000200000012790211D8
:10791000192A0F180A000000F1590000FD24000088
:1079200041460100BD350211D1550211452A02110F
:10793000C1330211010F021115640211E50B02118E
:107940007D050211000000000000000054757961FF
:107950000056302E3400303030310067697468755D
:10796000622E636F6D2F7076767800544842320035
:107970000200000084790211292A282A272A262AAF
:10798000252A242A0A18303132333435363738392B
:10799000414243444546005048592B3632585850CE
:1079A0004C555330353034005B4861726420666159
:1079B000756C742068616E646C65725D0A004C526F
:1079C0002020203D203078253038780A0050432090
:1079D00020203D203078253038780A00505352203E
:1079E000203D203078253038780A00494353522012
:1079F0003D203078253038780A000000111302113C
:107A0000651302110000000002000000147A021148
:107A10006F2A6E2A1A18FB349B5F800000800010CA
:107A2000000000000000000047160211D12C0211D6
:107A30006B160211D9300211EF160211AF3002118C
:107A40006517021185300211B71702114D3202116C
:107A50001F1802114D320211511802110732021182
:107A6000651702113D300211DD170211E5310211D7
:107A70000000000000000000C3180211E5310211EF
:107A800025190211E92C0211052A042A012A002ACB
:107A9000022903280128002801180018000000000E
:107AA000000000000000000000000087010102014A
:107AB00002010102010203030401030101010101AA
:107AC0000303020103000D000E001000110013005B
:107AD0001401070108010A010B011C011D02040227
:107AE00005020702080219021A021C021D03010303
:107AF000020317000201000504000807000B0A003A
:107B00001716001D1C010201010504010E0D0111D3
:107B100010011413011716011A19020201020B0AAF
:107B2000020E0D02111002141302171603050403AE
:107B30000807030B0A030E0D0001020307090A0BD5
:107B40000E0F101112141718191A1B1F20212200D2
:107B50005D5D0211195E02110000000002000000CC
:107B60009A7A021100000000456B0211000000002B
:087B700002000000987A0211E6
:107B780010B5F8F779FD06210020F8F703FE032079
:107B880000F0BAFAC022042192004020F8F71AFE49
:107B98000223FE21034A4020F8F7C6FDF8F7B2FD9C
:107BA80010BDC046DE61FF1FF7B50F490F4B0A68CD
:107BB80004001A4084235B0013430B60030003276F
:107BC8001033019300252E00112000F09DFA084B78
:107BD8001B683B40AB4002351E43202DF4D1019B6E
:107BE80040C4A342EED1F7BD5CF0004000FEFEFFAA
:107BF80064F000408022F8B5944C954BD2000021E7
:107C080020001C6000F088FA924B1A786E23002A34
:107C180000D01133E3620A2323658F4B18788F4B0A
:107C2800A0630138E361C3B2032B01D81023236298
:107C38008B4B37226361C823DB00A361894B362154
:107C48001A6008233B26884D0F3AE1632364626477
:107C5800E967864D0439E967854D2E60854D0636FE
:107C68002B60854D2A60854D2E60854D083E2E601F
:107C7800844D1B3E2960022583490B6083490A60B5
:107C880083490D604221834D2960834D2E60834DC9
:107C98002B60834D2A600525824A1560824A11604F
:107CA800824A18311160824A13603C22814B1A6063
:107CB800AF23DB002360804B2363032805D800F043
:107CC8003BFA34023638152363609623FA225B00A8
:107CD800A360E360C8332361784E794B9200A664B1
:107CE8001A606262774A0225A26273227649E265C7
:107CF8006D3A6265A2650232E1645A60656696254E
:107D0800AD00A566626709250022E566A2676F4D8A
:107D18006F4A704F2567E267396003280FD86E4FA6
:107D28006E4900F009FA86088A8E1023CCE70E23E4
:107D3800CAE70C23C8E71A20386007300860FA2021
:107D4800674980000E6067490860642066490860DA
:107D580066495F3808606649033808606549C63077
:107D680008600021644801603820986063485A66BA
:107D7800586463489A64D861962080001862614804
:107D88009A675862F538FF3898621E205E4AD866AE
:107D9800DD651D6619675967DA67BE235B4A5B00B4
:107DA800E25081315A4BFF31635004316250C42292
:107DB8005200A350FA2304325B00A3500432A350AC
:107DC800544B554A1360554B554A1360554B564A08
:107DD8001360564B564A1360564B574A1360574B1D
:107DE800574A1360574B584A1360584B584A136008
:107DF800584B594A1360594B594A1360594B5A4AC0
:107E080013605A4B5A4A13605A4B5B4A13605B4BD8
:107E18005B4A13605B4B5C4A13605C4B5C4A1360C3
:107E28005C4B5D4A136000F05FF9012000F04CF9EB
:107E3800F8BD14203860043080E710203860033023
:107E48007CE70E203860023078E7C0460004FF1F48
:107E58007464FF1FBC44FF1F4A0AFF1F3A07000053
:107E680080C3C9018C04FF1F0804FF1F0404FF1FFF
:107E7800BC04FF1FC004FF1FC404FF1FCC04FF1F66
:107E8800C804FF1FD004FF1FD404FF1FD804FF1F1E
:107E9800E004FF1FDC04FF1FE404FF1FE804FF1FCA
:107EA800EC04FF1FF404FF1FF004FF1F9004FF1FE2
:107EB8009404FF1F9804FF1F9A02000050C300009B
:107EC800FC04FF1F6A180000280A0000204E00006A
:107ED80088130000F009FF1F9C04FF1FA004FF1F68
:107EE800A804FF1FF804FF1FA404FF1FAC04FF1F12
:107EF800B004FF1FB404FF1FB804FF1F00400011A7
:107F080068100000C4090000DC05000040420F00B2
:107F180010270000FD1BFF1F0801FF1FFD2EFF1F7C
:107F28009003FF1F4532FF1FA801FF1FDD30FF1F11
:107F3800AC01FF1FD91FFF1F1801FF1FF51FFF1FEF
:107F48002C01FF1FA121FF1F3001FF1F491FFF1F29
:107F5800FC00FF1FC128FF1F9C01FF1F892CFF1F6A
:107F6800F800FF1FD918FF1F5801FF1FD127FF1F57
:107F78000802FF1F3925FF1F8400FF1F4525FF1F2B
:107F8800B400FF1F491EFF1F2002FF1F011FFF1F14
:107F98008800FF1FC11DFF1F4C00FF1FF7B50B0C0A
:107FA800FF270122009300233C001E001D00944679
:107FB800019089B262469A4010000840184136186C
:107FC800B6B2FF2F02D1012E00D19FB20098024015
:107FD8001A41AD18ADB2FF2C02D1012D00D19CB2CF
:107FE8000133102BE6D10320012E07D1012D04D136
:107FF800019B2401E4191C700138FEBD102EFCD130
:108008000238102DF9D00230F7E710B5064C237866
:10801800002B07D10548FFF7C7FD0548FFF7C4FD4A
:108028000123237010BDC0463464FF1F4864FF1F3E
:108038003864FF1FF0B58BB00D00012301901029A3
:1080480036D8FFF7E2FF00231A001B48C15C013352
:108058005218102BFAD1023B002A29D0174B184C82
:108068001F68002306A9E25C1600FA5C56405E54BD
:108078000133102BF7D102AA00F02EF82A0002A92A
:10808800019800F061F800F04FF823681B1823608E
:1080980000F04AF863681B18636000F045F8A368AD
:1080A8001B18A36000F040F8E3681B18E360002386
:1080B80018000BB0F0BDC0464864FF1F5C43FF1FAB
:1080C8003864FF1F0000000001B40248844601BC68
:1080D800604700BF456B010001B40248844601BCFB
:1080E800604700BFC53F000001B40248844601BC98
:1080F800604700BFADAE000001B40248844601BC31
:10810800604700BFED3AFF1F01B40248844601BC36
:10811800604700BF0189000001B40248844601BCE1
:10812800604700BFB70E000001B40248844601BC96
:10813800604700BFC95C010001B40248844601BC25
:10814800604700BF113CFF1F01B40248844601BCD0
:08815800604700BFE94C010083
:020000041FFFDC
:100000000000000011050211187902111479021183
:10001000C861FF1F00000000000000000000000099
:1000200000000000000000000000000000000000D0
:1000300000000000000000000000000000000000C0
:1000400000000000000000000000000000000000B0
:1000500000000000000000000000000000000000A0
:100060000000000000000000000000000000000090
:100070000000000000000000000000000000000080
:100080000000000000000000000000000000000070
:100090000000000000000000000000000000000060
:1000A0000000000000000000000000000000000050
:1000B0000000000000000000000000000000000040
:1000C0000000000000000000000000000000000030
:1000D0000000000000000000000000000000000020
:1000E0000000000000000000000000000000000010
:1000F0000000000000000000000000000000000000
:1001000000000000000000000000000000000000EF
:1001100000000000000000000000000000000000DF
:1001200000000000000000000000000000000000CF
:1001300000000000000000000000000000000000BF
:1001400000000000000000000000000000000000AF
:10015000000000000000000000000000000000009F
:10016000000000000000000000000000000000008F
:10017000000000000000000000000000000000007F
:10018000000000000000000000000000000000006F
:100190005D34FF1F4D33FF1FC166010000000000EA
:1001A000000000000000000000000000000000004F
:1001B000000000000000000000000000000000003F
:1001C000000000000000000000000000000000002F
:1001D000000000000000000000000000000000001F
:1001E000000000000000000000000000000000000F
:1001F00000000000000000000000000000000000FF
:1002000000000000000000000000000000000000EE
:1002100000000000000000000000000000000000DE
:1002200000000000000000000000000000000000CE
:1002300000000000000000000000000000000000BE
:1002400000000000000000000000000000000000AE
:10025000000000000000000000000000000000009E
:10026000000000000000000000000000000000008E
:10027000000000000000000000000000000000007E
:10028000000000000000000000000000000000006E
:10029000000000000000000000000000000000005E
:1002A000000000000000000000000000000000004E
:1002B000000000000000000000000000000000003E
:1002C000000000000000000000000000000000002E
:1002D000000000000000000000000000000000001E
:1002E000000000000000000000000000000000000E
:1002F00000000000000000000000000000000000FE
:1003000000000000000000000000000000000000ED
:1003100000000000000000000000000000000000DD
:1003200000000000000000000000000000000000CD
:1003300000000000000000000000000000000000BD
:1003400000000000000000000000000000000000AD
:10035000000000000000000000000000000000009D
:10036000000000000000000000000000000000008D
:10037000797202110000000000000000000000007F
:10038000000000000000000000000000000000006D
:10039000000000000000000000000000000000005D
:1003A000000000000000000000000000951AFF1F80
:1003B000000000000000000000000000000000003D
:1003C000000000000000000000000000000000002D
:1003D000000000000000000000000000000000001D
:1003E000000000000000000000000000000000000D
:1003F00000000000000000000000000000000000FD
:08183800000000204118FF1F11
:10184000024981F3088802F0BFFA0000000000207E
:1018500010B502F0E9FA072804D0122808D00228AF
:1018600008D010BD044A0420136B01331363F8E75A
:101870000220F6E71420F4E73465FF1FF8B50700EF
:101880000C0026002500503630785135002804D150
:101890000300287058342370F8BD2978CA00481E08
:1018A0008141A3183800A25C5B68C9B2FFF7D0FF82
:1018B00000280DD12B78DA00A218013350602B706C
:1018C0003378044A013B3370136A01331362D8E75B
:1018D0000123DFE73465FF1F5C234343074910B54D
:1018E000C9180B0058331B78012B05D1FFF7C6FF31
:1018F000034A936A0133936210BDC0466865FF1FB7
:101900003465FF1F10B502F067FB064A0121130082
:1019100010CB4942D967044B136002F08DFA2000C6
:1019200010BDC04600E100E01000100010B504003A
:1019300002F052FB024B1C6002F07EFA10BDC04662
:1019400000E100E010B5040002F046FB4021094A26
:10195000200013688B43136002F076F901F060FDFC
:101960000022054B01201A60044B04321A6002F079
:1019700013FBFEE71CF00040C4F00040C0F0004044
:10198000431E5A425341A022F0B5D2015B4213409C
:10199000154D164A40019B182A18127E8BB00191F2
:1019A000002A1BD01A000832D46F0022E6B206AF1C
:1019B000E4B294420EDC2818C369002B08D00199C8
:1019C00002AA117106AA049202AA167303A89847E4
:1019D0000BB0F0BD1978B9540132EAE71A7D1A78D4
:1019E00006AB01261A70E6E7F467FF1F00400040CF
:1019F000F0B5254B04004001C25C85B0002A2BD015
:101A00001A18117E002927D0917E002924D011793F
:101A1000022921D11689D788D168F51BADB22A1CBD
:101A2000102D00D9102292B2BE4217D118180123EE
:101A300003710023C269C38003819A4206D06846BD
:101A4000032103730171029301A890470820002C21
:101A500000D0192001F030FC05B0F0BD013C65421A
:101A60006C41A0256442ED012C40084D1B186419FF
:101A7000074D0633013A92B2AA42EDD01888461CAF
:101A80001E80085C2070F5E7F467FF1F00400040EF
:101A9000FFFF00000F220E4B10B59868104002386F
:101AA0000A280BD802F0B4F80D0A0B0A0A110A0A28
:101AB0000A0A060002210020FFF762FF10BD012183
:101AC000F9E70020FFF794FFF8E7DB6FF6E7C04681
:101AD000004000400F220E4B10B5986810400238AD
:101AE0000A280BD802F094F80E0A0B0A0A120A0A06
:101AF0000A0A060002210120FFF742FF10BD012162
:101B00000800F9E70120FFF773FFF7E7DB6FF5E760
:101B10000090004013B5334C2378072B3DD8324B4F
:101B20001A78324B002A39D18022196852020A43AE
:101B30001A60252001F026FF20232D4A11680B434F
:101B4000802113606B460422C905086807331042E0
:101B500028D080210422C905C86810422ED08021D7
:101B60002020C905CA688243CA6014221A701A78F4
:101B7000002A2FD18021C905C86820320243CA60DB
:101B800014221A701A78002A28D11A4B1A7D22784A
:101B90005A601D221A705932DA6013BD1A6816494C
:101BA0000A40C5E7086802430A6014221A701A78CE
:101BB000002ACED01A78013AD2B2F7E7C8680243B9
:101BC000CA6014221A7019784A1ED2B21A700029FB
:101BD000F9D1C4E71A78013AD2B2C7E71A78013AC4
:101BE000D2B2CEE7F443FF1FBC44FF1F3CF00040DD
:101BF000EC43FF1F00200040FFFFFEFF564B70B577
:101C00001B68012B03D1554A936D0133936502F094
:101C1000D3F9534B534A1860534B544C1A60012369
:101C2000534A1360534A13602378002B06D00622D0
:101C30005149524802F030F800232370504A514B6A
:101C400010681B78C1B2002B0ED14F4CC0B2237864
:101C50005BB2002B4FDB237824785BB264B21B04A9
:101C600024021B191B1813600B1C50294ED950233A
:101C7000464A47491078DBB2FF2202284BD1086858
:101C8000444C454D267890432A78964254D9227880
:101C900024782E78023B5D10A31B6B435201D31AAC
:101CA00010335B111843086002F0BEF9031F012BCB
:101CB00045D83A4B1B78002B06D0394B1B78002BAC
:101CC00002D0002002F040F8A122364B9200997811
:101CD000354B4A431B689B18832292009B181B7844
:101CE000033B012B03D8AF20400001F0E5FF0122A8
:101CF0002E4BDA8270BD237824785BB264B2FF3356
:101D0000FF341B0424021B190138ABE7CAB2022AB4
:101D1000AED20223ACE70868254C264D26789043C6
:101D20002A78964208D9227824782D78023B5B10D5
:101D3000641B63435201B2E72378DBB2B2E70228A7
:101D4000D5D11D4B1B78013B022B03D91B4B1B78B4
:101D5000022BCCD16C20C8E79809FF1FFC0FFF1F96
:101D60006C64FF1FFF3F0000141003407064FF1FEE
:101D70000C10034000100340D50BFF1F7211FF1F12
:101D8000B40003408C09FF1F680AFF1F490AFF1FA8
:101D900094000340460AFF1F470AFF1FF908FF1F70
:101DA0002209FF1F300DFF1F3409FF1FBC0BFF1F4F
:101DB000440AFF1F450AFF1F1C09FF1F2309FF1FBD
:101DC00010B502F069F80022014B1A8010BDC04620
:101DD0006864FF1F10B502F017F9A121054A8900B8
:101DE0009478054A61431268044B5218528C1A8049
:101DF00010BDC046300DFF1F3409FF1F6864FF1F70
:101E000010B50D4B0D4A9978A1239B004B431268E6
:101E1000D218531DD97F0A4B1B88994209D2441C02
:101E200007D0C82805D0D2695B1A5A43054B5343E3
:101E3000C01801F099FF10BD300DFF1F3409FF1FBE
:101E40006864FF1F7102000070B5244D2B68002BE1
:101E500028D002F059F82B68D8402B680400002BDA
:101E600027D002F0A1F82B68D8401D4B1D4A997865
:101E7000A1239B004B431268D118D25C91239B0095
:101E8000002A20D0CA580132CA50174B17491B6884
:101E90000868834214D3D23B181A012A1AD0144B73
:101EA000186070BD02F030F8124B196802F064F946
:101EB000D3E702F079F80F4B196802F05DF9D4E727
:101EC0000D495B18E8E7CA500C4B1B68DB68E41847
:101ED000201AE4E7F530FF30E1E7C0461C08FF1F99
:101EE000300DFF1F3409FF1F9C09FF1F6C64FF1F8B
:101EF000A009FF1F1808FF1F2DFF3F007464FF1F7C
:101F000070B504000D00282916D10300A433C2883F
:101F10001B889B1A0B4A9BB293420DD906006A3666
:101F200005223100653001F0FFFE002804D13100A8
:101F3000200001F0D1FE70BD2900200002F0ACF8B5
:101F4000F9E7C046FE7F0000F8B50400012002F06A
:101F5000E3F801F0B9FF174A174910600968030058
:101F60001648174E01601748776805680020AF4291
:101F700001D27068281A144D091928601348C162EB
:101F8000A421446A49032143416211490978002987
:101F900005D010490978022902D10F3B1360F8BD22
:101FA000012901D1083BF9E7032901D1053BF5E7F8
:101FB000033BF3E7E408FF1F28F00040340AFF1F4B
:101FC00028100040180AFF1F1C0AFF1F00F00040E5
:101FD0001C09FF1F4A0AFF1F70B580241025E40565
:101FE000A3682B43A36001F0DFFEA368AB43A360AB
:101FF00070BD0000F7B5160080221C001023D2052A
:102000000191916805000B43936000225A4BD73031
:102010001A6001F051FF9D232A002F009B00EB580E
:10202000CA3201210092FC37002B01D00021009A16
:10203000386801F029FE2900009BCB311A784F4BFC
:10204000D3351A604B780A781B0213438A7812043E
:102050001A43CB781B061343494A1BBA13604B79CA
:102060000A791B0213438A7912041A43CB7931008F
:102070001B061343434A1BBA13606B782A781B0272
:102080001343AA7812041A43EB781B0613433E4A03
:102090001BBA1360019A330213433C4A13603C4B52
:1020A00022001B1B9C4603293DDCB3089A00130049
:1020B0005142B21A032A46D1354AE018511A8278A1
:1020C0004078120400020243E05C043302430A60D9
:1020D0000022FF2B4BDDF0222E4B12011A600F2243
:1020E0002D4B1A602D4A1368002BFCD00023224A86
:1020F00027491360091B321D0B191B68043A180A83
:1021000023706070180C1B0EA070E3700434002A5A
:10211000F2DC802210213B68D20501333B609368DA
:102120008B439360F7BD6346D578981893782D0656
:102130001B042B43157804392B43557804322D02A8
:102140002B430360AFE7022A0AD1114AE05C511A1F
:10215000E2185278120202430A6004339BB2B7E7D6
:10216000012AB5D10A4A521AE15C1160F5E7084923
:1021700059180A600433ACE7000004403C000440F6
:102180003800044034000440300004400C00044097
:102190000001044004000440100004401400044006
:1021A000F7B5150080221C001023D205009191681C
:1021B00007000B4393600023654AD730136001F09A
:1021C0007BFE9D233E009B00F9583B00CA3632003F
:1021D000FC33002900D07FE0586801F055FD39003C
:1021E00032785C4BCB311A604B780A781B02134370
:1021F0008A78AC4612041A43CB78281D1B06134379
:10220000554A1BBA13604B790A791B0213438A792A
:1022100012041A43CB791B061343504A1BBA1360AE
:102220004B7A0A7A1B0213438A7A12041A43CB7A36
:1022300021001B0613434A4A1BBA1360009A2B0263
:102240001343484A13602200474B1B1B0093009B1B
:10225000CE785B1801938B7836061B0433430E78D7
:10226000043833434E78043136023343019E3360E1
:102270000328ECDC0321A808431C9B0029408000B4
:1022800003292BD13849E5185E18A9786D78E35CED
:1022900009042D022943194331600300083300214A
:1022A000FF2B2DDD314B324919600F21314B196065
:1022B000012327490B60304B19680029FCD0062107
:1022C0001B680B40042B20D080220020D20593688D
:1022D0000A318B439360FEBD01217DE7022908D1BD
:1022E00021495D18E1184978E35C09021943296026
:1022F000D3E70129D3D11C495918E35C0B60CCE723
:102300001948181801600433CAE7002310490B600C
:102310006346002B0CDC3B00FC335A681021013271
:102320005A608022D205936801208B439360D2E7E4
:10233000009B9B181B68190A13705170190C1B0E17
:10234000D37004235B4291709C440432E0E7C046A2
:10235000000004403C0004403800044034000440C5
:10236000300004400C00044000010440040004401C
:10237000080F0000100004401400044070B5061E51
:1023800019D00222614B9B799343012B13D1604BEF
:102390001A78FF2A0FD15A78FF2A0CD19A78FF2A8F
:1023A00009D1DA78FF2A06D11A79FF2A03D15B799D
:1023B000FF2B00D1A7E0574B0C201A78012A08D038
:1023C0000022554D1A702B781A00093A042A01D8B8
:1023D000212070BD5A1F012AFAD94C4CA07B042839
:1023E00000D990E0A279032A00D98CE0821E012A4C
:1023F00003D862881F2A00D885E0002E61D0012E04
:1024000000D080E0A288012AE2D0002B0AD1013856
:10241000032803D801F0FCFB151D19151F202E7091
:1024200001F0FAFD2B785A1E032A16D800253B4BE3
:102430001D602823237501F01FFEA8422ED0A58021
:10244000C6E7022320202B70EAE7042322202B700A
:10245000E6E7032321202B70E2E7073B012BB7D8E7
:102460002F4B1B68DB6A9B06B2D52E4B1A78002ACD
:10247000AED1A27B911E012901D9002AA8D1022246
:1024800080211A702823284D89012878237501F0AE
:1024900073FD80212878890101F0F6FC0123A380D7
:1024A000224B1B78002B0AD0FA228021204B92006D
:1024B0001B8809025A431C4B187801F0CDFD0020FF
:1024C00087E701F089FD2B78A680073B012B06D911
:1024D00018482E7001F0E8FC1E2001F09DFD114B04
:1024E000114C1A78002A06D0802100222078890118
:1024F0001A7001F041FD01F09FFC80212078090253
:1025000001F03AFDDBE7122063E7C046A60BFF1F90
:102510006B09FF1F1A09FF1F1C09FF1F4809FF1F36
:102520007464FF1F2309FF1F1B09FF1F2109FF1FE1
:102530002C09FF1F0010004010B5002901D001F048
:10254000CBFD10BDF7B5604B01919978A1239B009D
:102550004B435E4A060014681022E418D6235B0041
:10256000E0583623FF33E35C00279343222B41D10D
:10257000574B0F3A1A600760012501F045FC019B9B
:102580001880E8235B00E35C002B01D0B34258DDE8
:102590000023504FFB70AD33FF33E3581A68002A15
:1025A00003D09B88DB439B071DD03823FF33E35CBC
:1025B000002B18D09B235B00E35C002B13D1D1339D
:1025C000FF33E35CB3420EDAA4235B00E15AE01868
:1025D000090A023101F090FD23000122FE33013E81
:1025E00001351A87FA70E8235B00E35C002B2AD0E0
:1025F000A8B2FEBD03683D00002BBED08188043028
:10260000090A023101F078FDD6235B00E3581F6010
:10261000B2E72300B133BA00FF33985801378188FD
:102620000430090A023101F067FDE8235B00E35C36
:10263000BB42EEDCE822F61AED1800235200A35448
:10264000A6E70027F1E7200001F0FEFB00281FD0DD
:10265000002E1DDD7319882647190193B60020004E
:1026600001F072FC5A3080002018406801358188E2
:102670000430090A023101F03FFD200001F0B4FCF2
:10268000A3590133A351BD4202D0019B9D42E6D123
:10269000114BE35C002BABD095239B00E35C002B3C
:1026A000A6D00E4BE15A0029A2D00D4AA35C994254
:1026B00002D90133A3549BE700231A212000A3541D
:1026C00001F062FC94E7C046300DFF1F3409FF1F84
:1026D00000140340E010FF1F5A02000072020000C5
:1026E0005E020000F8B51D4B1D4F1A78002A10D16C
:1026F000BA7B002A02D101321A7003E0032AFAD011
:10270000022AF8D001F0B8FC00220120154B1A7003
:10271000F8BD154B154D1C68154B9E7801232B7089
:102720002878C0B200F0DAFCBB7B002B0BD101F0A3
:1027300083FAA1239B007343E41883239B00E418CE
:1027400023782B70E4E7032B02D101F0BDFAF0E708
:102750000020022BDCD101F017FBEAE71C09FF1F68
:10276000A60BFF1F2309FF1F3409FF1F490AFF1F84
:10277000300DFF1FF0B587B00EAD2F780FAD2D785F
:102780000593AC46634614000E4D0CAA12782E78C1
:1027900003930D9B009201932200059B029701F089
:1027A000FBFA2E70012C01D0042C08D1802206499E
:1027B0008B889343054A1278D20113438B8007B06C
:1027C000F0BDC0461C09FF1F6C11FF1F7809FF1FD9
:1027D0000B001B3B70B504003020E02B0DD813001C
:1027E000E025493BFF3B9BB2ED00AB4205D8034BD4
:1027F000200019825A8201F077FB70BD8410FF1F00
:1028000010B501F0D9FB054B00205B68052B04D9FE
:10281000034A5268D20200D4980810BD001000404C
:10282000FCE100E070B501F0D7FB0D4B1B68FC33F9
:10283000DC691D6AFFF7E4FF6419844204D2094B86
:1028400001241B68002B07D004220024064B1A70B9
:10285000064A93690133936101F0EEFA200070BDDE
:102860007464FF1F9809FF1F2309FF1FFC0FFF1F40
:1028700070B50C4D2B68FC335C6A01F0ADFBFFF7C3
:10288000BFFF2B680025FC339B6AE318834204D208
:10289000054B1B68AB4200D1051B01F0CDFA2800A7
:1028A00070BDC0467464FF1F9809FF1F034B10B52D
:1028B0001B68002B00D0984710BDC0465C03FF1F6B
:1028C000F0B587B001F02EF9FFF7F0FFCA4BCB4C03
:1028D00004931B78022B45D1C94B1B68186A01F081
:1028E0001BFCC84BC84A1A60C84BC94A1A60A022D0
:1028F000C84B52001A60049B187801F0B5FBC6491A
:10290000C64801F0A9F9C649C64801F0A5F9102248
:10291000C54BFF201A60802252031A608022920366
:102920001A60802212041A6001F00EFA012001F0F0
:10293000ABFBFA20400001F0FFFA582001F0BCF98F
:10294000BA4801F049FA012001F0BEFB072001F06E
:102950008BFA2268B64B1A4084235B001343236032
:1029600007B0F0BD01F088F9B24E0290322001F0BC
:10297000D3FB33681B0629D43C2001F0CDFB0F208C
:1029800001F0CAFB9C4B1B78012B00D11EE1802279
:102990003368A94D134200D0A7E02B6803201343EE
:1029A0002B6001F0B9FB01F067F9029B0299C31A91
:1029B0005A1E814200D81A00A04B1A60904B196829
:1029C0001E2353439E4A9B18CB618AE701F054F9BA
:1029D00080239C4ADB02116803900B43136022683A
:1029E000934B994F1A40282313432360032001F08F
:1029F00093FB03203D6801F08FFB3B680320DB0362
:102A0000DB0B009301F088FB3B68ED03DB03ED0B70
:102A1000DB0B8E4A0193AB18C22B30D8009B9B185E
:102A2000C22B2CD8019B9B18C22B28D8009B2A00B4
:102A30009D4200D21A00009B9D4200D91D00019BBF
:102A4000934200D21300019A954200D915005B1BF6
:102A5000122B14D80C22336814209343336033684C
:102A60007B4A1340336001F057FB08213B68226822
:102A7000DB038A432260774ADB0B13607FE7032086
:102A800001F04AFB3B68DB03DB0B059301F0F4F834
:102A9000039B0399C21A531E814200D813006E4A49
:102AA00093421BD9FF23356869492D0A1D403268BE
:102AB0006B1C1B060A401B0C134333600C2332684B
:102AC00000209A43083B1343336001F045FB634801
:102AD000634BA840984206DCFEF734FF019B009D43
:102AE0000093059B95E75F48F6E700235E4F554A44
:102AF0003B6080231168DB020B43136080222B684C
:102B0000032013432B6001F007FB3B6805260133CC
:102B10003B6080232A685B0213432B602268444B8E
:102B200003201A40514B1343236001F0F5FA0821AA
:102B3000454B1A682368D2038B432360454B023907
:102B400000931B68D20B4B439A420CD89B1A3B2B29
:102B50000BD8236846490B4023602B680B402B6041
:102B6000444B1A601FE7D31AF1E7013EF6B2002E7C
:102B7000D4D123683E4A134023602B6813402B6056
:102B80003B68042B07D9BFF34F8F3B4B3B4ADA60BE
:102B9000BFF34F8FFEE780222B68032093432B6007
:102BA00001F0BAFA2268224B03201A40282313436B
:102BB000236001F0B1FA244B009A1B68DB03DB0BA6
:102BC0001360082223689343236097E707222C4D64
:102BD0002B681340012B02D1002001F045FAAB68AD
:102BE000284A02201340AB6001F096FA8023AA68BD
:102BF0005B001343AB60D6E64A0AFF1F5CF000405F
:102C00007464FF1F000003400180063DBC000340C8
:102C100034080000A40003407102000014100040BA
:102C2000FFFF3F002810004000E100E03075000089
:102C300000FEFEFFC4F0004044F000405C64FF1F53
:102C40007206000040F0004064F0004091FCFFFF7D
:102C5000FF00FFFF6464FF1FE30C0000E88000003A
:102C60005F361E0060361E005843FF1F280001001B
:102C7000FFFFFEFF6064FF1F00ED00E00400FA05A7
:102C80003CF00040FFFEFFFF664E336888331B6850
:102C900083F3088801F050F8634B644A1B68934241
:102CA00007D0002001F058FA0221614A13688B43D3
:102CB0001360FFF705FE5F4B5F4C1878C0B201F060
:102CC000CBF80023A3600233A3605C4B0120236098
:102CD00001F022FA0323A36000F0CEFF040001F00C
:102CE0006BF9050000F0C8FF554B186001F034F98E
:102CF000544B1968621A531EA14200D2130080225D
:102D0000D203934201D39B029B0A3268D16AC9075E
:102D100000D475E04C491C0C09689BB24C435943E4
:102D20002402090A641803274849FC3293680A6898
:102D300047489B1A474A484E126848499B183F4AE1
:102D400034609A183B400193036892089C46019BAB
:102D50000A6063440360042B03D901323B400A60DC
:102D600003600B683E49E418200001F005FA3D4F6E
:102D70003B493B68C3183B602000019300F0B4FF5F
:102D8000394C2068081836492060884205D9019BD3
:102D900001333B6000F0A8FF216001F0B5F9334B2F
:102DA0001B78002B0ED001F007F93168304B4A1B1D
:102DB0001B6812189A4230D2591A4919091A2D481B
:102DC00000F04AFF2C4C237A002B0FD001F0F4F8CE
:102DD0003168E3684A1B1218934221D9591A4919DC
:102DE000091A264800F038FF0023237200F0C4FFC0
:102DF000022001F011F9002001F0AEF900F0F4FF1B
:102E0000DC0199000234641A5900641A09214B4309
:102E10008033CB40A408E41885E7FA218900CEE787
:102E20001749DEE77464FF1F0C0AFF1FB641210338
:102E300010000040490AFF1F14100040C4090000A0
:102E4000100AFF1F340AFF1F380AFF1F200AFF1F46
:102E5000280AFF1F1C0AFF1F5864FF1F240AFF1FB8
:102E6000710200006008FF1F2C0AFF1F1C09FF1FD2
:102E7000E408FF1F00100040740BFF1F3C100040CF
:102E8000DC050000044B10B51B68002B01D09847EF
:102E900010BD01F031F8FBE78002FF1F044B10B5B5
:102EA0001B68002B01D0984710BD01F025F8FBE707
:102EB0008402FF1F044B10B51B68002B01D09847FC
:102EC00010BD01F019F8FBE78802FF1F044B10B595
:102ED0001B68002B01D0984710BD01F00DF8FBE7EF
:102EE0008C02FF1F044B10B51B68002B01D09847C4
:102EF00010BD01F001F8FBE79002FF1F70B501F073
:102F00005BF8514B1860042001F086F801F09CF842
:102F10000400C30702D401F0C7F870BD00224B4B78
:102F20001A604B4B1878013804282CD800F070FE3A
:102F300003231B1F2700200000F05EFF0128ECD0B8
:102F4000444C2378042B71D100F0D6FE002806D023
:102F500000F062FF582000F0AFFE02232370032030
:102F600001F05AF8D9E7200000F0B6FFE6E72000AC
:102F700000F0CAFEE2E7200000F0CEFFDEE720000E
:102F800001F022F8DAE701F04FF80500012808D136
:102F9000314B1B78053B012B03D82000FFF772FF54
:102FA000CEE72C4B1B78022B01D0052B20D1022D14
:102FB00028D12A4B9B7BAB431CD12000FFF76EFF2F
:102FC000254B18780128BBD16405B9D423492522A3
:102FD0004B7B034205D1233A13405A4253412633D7
:102FE0001A000B7D9342ABD9322001F0BDF8A7E760
:102FF000022D07D1184B1B78052B11D12000FFF7AC
:1030000059FFDDE7012D0BD1012B03D12000FFF784
:103010005DFF95E7062B03D12000FFF763FF8FE7E5
:10302000200000F069FF022D8AD1C9E7032B04D1EB
:103030000B4B987C00F0E0FF91E7072B8FD1094BF9
:10304000987B01F071F88AE79C09FF1F9809FF1F20
:103050009009FF1F2309FF1F1C09FF1FA60BFF1F5D
:10306000BC0BFF1FD40BFF1F0A4B0B4A13600B4B0B
:103070000B4A13600B4B0C4A13600C4B0C4A136049
:103080000C4B0D4A13600D4B0D4A13600D4B0E4A4D
:10309000136070477527FF1F4000FF1F7128FF1F37
:1030A000F401FF1F2528FF1FF001FF1F7D23FF1FD5
:1030B0004800FF1FE526FF1FF801FF1F011EFF1F2D
:1030C0005402FF1FD51DFF1F6C00FF1F10B500F03D
:1030D00087FD10BDEFF30380704700008023F7B534
:1030E0009C46264B264F01932649274A274D284CBC
:1030F000284B02281AD1604638600868264E3040B6
:10310000802636033043086001990978002909D1E7
:103110001660224A2A60224A2260E02219689143FE
:10312000A03A1BE08021C9021160F2E766463E60CA
:103130000F68194E3E408027FF023E430E60019902
:10314000097800290DD1176001280ED1154A2A608F
:10315000154A2260E02219689143C03A0A431A6076
:10316000F7BD802189021160EEE7E0210F4A02439A
:103170002A600F4A22601A688A43F0E74B0AFF1F51
:10318000E0000340D80003409000034000000340EB
:103190005000034040000340FFFFE3FF0280063D74
:1031A000804508220180063D80660822008006983E
:1031B00080550822F8B51E4B80261A68002014009E
:1031C0003440324232D11A681A4F32431A60012217
:1031D0003B68063093433B6000F09EFF0122164D92
:1031E0002B681E432E603B680A2613433B608027F2
:1031F000BF00124B1B683B4211D1013EF6B2FF2EBD
:1032000009D17E220E4B1C682B68E40B14409343BB
:1032100023432B6005E0082000F07EFFE9E7002E45
:10322000EFD180222B68600893432B60F8BDC04625
:10323000C4F000405CF0004018F0004068F000402E
:1032400060F0004010B500F04FFF01215820034A04
:1032500000F06AFEFFF7AEFF10BDC046600AFF1F18
:1032600010B578220021034800F026FF00F004FE8C
:10327000002010BD7C67FF1F70B5040000F0ACFE9D
:1032800000230C200B4A010059438D18515C002982
:103290000DD0A14208D1012300246B7000F04CFF37
:1032A00000F0CAFD200070BD01330A2BEBD11224BF
:1032B000F6E7C0467C67FF1F70B5040000F08CFE87
:1032C000002319001D000D4A1078002806D0A042E6
:1032D0000CD1557001310C320A29F5D1002B0AD1DD
:1032E00000F0CAFD00F0A8FD002070BD5078461E19
:1032F000B0411B18EEE700F01FFFF3E77C67FF1FEC
:10330000F7B504000C20002384460E4D0192674659
:103310005F43E85D7E19A04212D000280BD10A4B12
:103320009C4662461B7808331370019B70707C5575
:103330007160B360FEBD01330A2BE8D10320F9E7C9
:103340000720F7E77C67FF1F7867FF1F8021204B6E
:10335000C9051B6870B58B601E4BC1241A68012318
:10336000FF2013434B611C4BA4001A681B4B002524
:103370001A601B4B1A681B4B1A601B4B1A5982436D
:103380001A51C52292009C588443BF38204398505C
:103390009C58164804408020C001204398509858FB
:1033A000134C0002000A01439950124B1B78DB08B2
:1033B000AB4201DC002070BD2378002B06D0A3684F
:1033C000002B00D0984701350C34EEE71220F2E7CD
:1033D000F043FF1FEC43FF1FB0F000407467FF1F76
:1033E000B4F000407067FF1F00E100E0FF00FFFF46
:1033F0007C67FF1F7867FF1F030010B51F2809D8DF
:10340000072200201340072404490A78A2431343EB
:103410000B7010BD00230620F5E7C0467867FF1F3C
:10342000034A0449136800200B4013607047C046EC
:103430001CF00040FFFFC1FF054B06491B780A68DE
:1034400005485B0702401B0B134300200B607047CD
:103450007867FF1F1CF00040FFFFC1FF70B50C250F
:10346000FFF7EAFF0A4B1C780A4BE4086543ED18A6
:10347000002C01D1200070BD2B78002B06D06B688A
:10348000002B00D09847013C0C3DF1E71220F2E7F9
:103490007867FF1F7067FF1F07B50422074801A95F
:1034A00000F034F9019B013305D18023044ADB0489
:1034B00011680B43136000200EBDC0461C1800119C
:1034C00014F0004007B500F087FD80220821D205E6
:1034D000936A0191002B01D10739916202210C4AB4
:1034E00011600199481E01900029FAD10331116041
:1034F000053101910199481E01900029FAD111600E
:10350000002B02D18022D205936200F095FC07BD0A
:1035100000C00040F0B505002026184B87B004938A
:10352000049B002B03D11124200007B0F0BD002123
:1035300002220B0001910091052000F03DFC0223C6
:103540000F490A681A42FCD10596059C631E059333
:10355000002CFAD10B4A1368002BFCDA0F276F44BA
:103560000121380000F068FD3B782B42DCD00520BB
:1035700000F0D2FD049B013B0493D1E7FFFFFF075E
:1035800090C8004000C80040F0B52D4C89B02378A9
:10359000002B4FD1FEF7B6F902232A4F03903A6869
:1035A0001A42FCD120230693069B5A1E0692002B3A
:1035B000FAD1254E3368002BFCDA0120FFF7AAFF71
:1035C000011E02D0112009B0F0BD030003220190BA
:1035D000009005AD9F2000F0EFFB0321280000F0D4
:1035E0002BFD02233A681A42FCD120230793079B44
:1035F0005A1E0792002BFAD13368002BFCDA012007
:10360000FFF788FF0028DDD10398FEF78FF9AA782D
:103610006B7811041B020B4329780B436360130082
:10362000113B0A49052B07D801239340A3600B6087
:10363000012323700020C6E780231B03F6E7C04662
:10364000D843FF1F90C8004000C800409808FF1FE3
:103650001E4B30B55A6818781D4B85B0D3185942A7
:103660004B4101210093002300F076FB194B1A4ACD
:1036700002259A6300221A6510325A658022C421FD
:103680009D65164B1648D202DA6789004258154BE1
:1036900080241A4080231B04134343506423412099
:1036A0000393E40500F06EF9402000F06BF96562C9
:1036B000039D6B1E0393002DFAD103236362FFF772
:1036C00001FFA562FFF760FF05B030BDE443FF1FB7
:1036D00095FFFEF700C80040050001FF04E100E08F
:1036E00000E100E0FFFF00FF10B5064B18705960C5
:1036F000FFF7AEFF00211320034AFFF701FE002071
:1037000010BDC046E443FF1F5136FF1FF0B5040053
:1037100085B003920291FEF7F5F8882263035B0BF4
:1037200052051A438023DB059D6A8023274F0092B0
:10373000BA68002601901B039A420CD9F823260090
:103740001B041E401C4206D08022214B52025E62A6
:1037500019680A431A60002D0BD100F03DFC0222CB
:103760001C4B1A608023DB055A62013A9A6200F012
:1037700063FB0023039A934220D1002D0AD100F06D
:103780002BFC144B03221D608023DB055A629D62D3
:1037900000F052FB8023BA681B039A4208D9002E1E
:1037A00006D000220A4B0C495A621A680A401A6075
:1037B0000198FEF7BBF8002005B0F0BD009A029911
:1037C000D2181278CA540133D4E7C046D843FF1F39
:1037D00000C8004000C00040FFFFFEFFF0B587B00A
:1037E000029103920400FEF78DF8019000F0F4FBC3
:1037F000802302250122234EDB0535605D629A623B
:1038000000F01AFB204F3B682B42FCD1202304938D
:10381000049B5A1E0492002BFAD11C4D2B68002BDE
:10382000FCDA0120FFF776FE002802D0112007B055
:10383000F0BD2000039A029900F096FB02230400D9
:103840003A681A42FCD120230593059B5A1E059223
:10385000002BFAD12B68002BFCDA0120FFF75AFE6F
:10386000051EE3D100F0B8FB80230322DB053560A1
:103870005A629D6200F0E0FA0198FEF757F8E0B254
:10388000D5E7C04600C0004090C8004000C80040D6
:10389000F0B5802687B00400FEF734F8F605B36A69
:1038A00002250393029000F097FB0123244F3D6013
:1038B0007562B36200F0C0FA224E33682B42FCD12D
:1038C00020230493049B5A1E0492002BFAD11E4D10
:1038D0002B68002BFCDA0120FFF71CFE002802D029
:1038E000112007B0F0BD200000F016FA022301906D
:1038F00032681A42FCD120230593059B5A1E05927B
:10390000002BFAD12B68002BFCDA0320FFF702FE14
:10391000041EE5D100F060FB80230322DB053C6040
:103920005A629C6200F088FA039B002B01D1FFF7DA
:10393000C9FD0298FDF7FAFF6B461879D1E7C0463A
:1039400000C0004090C8004000C8004073B50500AA
:1039500005240B4AA3005B429B1819686B46DE1DC9
:10396000300000F0A1F9022804D133782B55013C36
:10397000EFD276BD052CFCD00128FAD10230F8E751
:10398000140900111F2807D8012380228340D20583
:1039900091680B43936070473F2808D80123802229
:1039A00020388340D20551690B435361F3E75F2808
:1039B000F1D80123802240388340D205116A0B439D
:1039C0001362E8E71F2807D8012280218240C90539
:1039D0008B6893438B6070473F2808D80122802171
:1039E00020388240C9054B6993434B61F3E75F2858
:1039F000F1D80122802140388240C9050B6A9343E7
:103A00000B62E8E71F2810D880230200DB05153A77
:103A10001968012A06D820229143196019680A43BF
:103A20001A60704701228240F6E73F2811D88023B0
:103A30000200DB05353AD968032A06D810229143E3
:103A4000D960D9680A43DA60EBE701222038824066
:103A5000F5E75F28E5D842238022181A413B8340CE
:103A6000D205516A99435162516A0B435362D8E7B8
:103A700010B50400012813D1A022184992050B6843
:103A80005B015B0913430B60154B164A1968114023
:103A9000154A0A431A60402219680A431A6010BD89
:103AA0000028FCD101000A2000F0DEF821000B20E4
:103AB00000F0DAF8C0220A4B920019680A4340214C
:103AC0001A601A688A431A60B022044912060B6809
:103AD0005B015B0913430B60E1E7C04614F0004053
:103AE0001CF000407F00FEFF80FD0100FA2110B5B0
:103AF0008900C00300F040FB00F00EFB10BD000089
:103B0000044B054A1A60054B1A600022044B1A60E8
:103B10007047C046140AFF1F841E0000380AFF1FAA
:103B2000C4F000400023034A1360034A1360034AB1
:103B30001360704754F0004040F1004044F10040F1
:103B4000002310B5184C8AB0009301932378012B01
:103B500027D06946012000F0F7FA002817D1009B12
:103B600012490293019B06AA0393114B02A81B68FA
:103B70000493104B1B68059300F016F910220E49B0
:103B800006A800F0D1F8002804D1FF2323700020FC
:103B90000AB010BD0123094A074902A8237000F0AA
:103BA00003F90120F4E7C0467864FF1F10290011D3
:103BB000082900110C290011202900117C64FF1F25
:103BC00013B501246946012000F0BEFA034B0094AE
:103BD0000193FFF7B5FF200016BDC046BB0B0000E8
:103BE00010B5FFF79FFFFFF7EBFF002802D0024B55
:103BF000984710BDFEE7C046E1A2000002B471463E
:103C000049084900095649008E4402BC7047C04625
:103C100002B4714649084900095C49008E4402BC5F
:103C20007047C04603B47146490840004900095A2C
:103C300049008E4403BC704701B40248844601BC6D
:103C4000604700BFE9F6000001B40248844601BCA9
:103C5000604700BFF9A6000001B40248844601BCD9
:103C6000604700BF2D6C010001B40248844601BCCE
:103C7000604700BFD557021101B40248844601BC19
:103C8000604700BF156B010001B40248844601BCC7
:103C9000604700BF2144000001B40248844601BCD3
:103CA000604700BFE94C010001B40248844601BCF2
:103CB000604700BFA57F021101B40248844601BCE1
:103CC000604700BF7912010001B40248844601BC7C
:103CD000604700BF75F8000001B40248844601BC8B
:103CE000604700BF85C1000001B40248844601BCA2
:103CF000604700BF090E000001B40248844601BCC1
:103D0000604700BF01D7000001B40248844601BCEF
:103D1000604700BF0534010001B40248844601BC7D
:103D2000604700BFA96F010001B40248844601BC8E
:103D3000604700BFCD4C010001B40248844601BC7D
:103D4000604700BFC9A9000001B40248844601BC15
:103D5000604700BFED6B010001B40248844601BC1E
:103D6000604700BFC56D010001B40248844601BC34
:103D7000604700BF8937010001B40248844601BC96
:103D8000604700BF7997000001B40248844601BC37
:103D9000604700BF19FA000001B40248844601BC24
:103DA000604700BF9D6A000001B40248844601BC20
:103DB000604700BFDD3F000001B40248844601BCFB
:103DC000604700BF496D010001B40248844601BC50
:103DD000604700BF8572021101B40248844601BCED
:103DE000604700BF8D11010001B40248844601BC48
:103DF000604700BF8552010001B40248844601BCFF
:103E0000604700BF0134010001B40248844601BC90
:103E1000604700BFCD0C010001B40248844601BCDC
:103E2000604700BF6DF6000001B40248844601BC43
:103E3000604700BFE927000001B40248844601BC86
:103E4000604700BF9DA9000001B40248844601BC40
:103E5000604700BF71B0000001B40248844601BC55
:103E6000604700BF8914010001B40248844601BCC8
:103E7000604700BFF90D010001B40248844601BC4F
:103E8000604700BFADAE000001B40248844601BCEB
:103E9000604700BF0D52010001B40248844601BCD6
:103EA000604700BF8D82000001B40248844601BC17
:103EB000604700BFC1A5000001B40248844601BCB0
:103EC000604700BF8944000001B40248844601BC39
:103ED000604700BFBD5C010001B40248844601BCDC
:103EE000604700BF0934010001B40248844601BCA8
:103EF000604700BF116E000001B40248844601BC57
:103F0000604700BFE917010001B40248844601BCC4
:103F1000604700BFE90B010001B40248844601BCC0
:103F2000604700BFF535010001B40248844601BC7A
:103F3000604700BF0167010001B40248844601BC2C
:103F4000604700BF8512010001B40248844601BCED
:103F5000604700BFD9B0000001B40248844601BCEC
:103F6000604700BFC166010001B40248844601BC3D
:103F7000604700BF9573010001B40248844601BC4C
:103F8000604700BFB352010001B40248844601BC3F
:103F9000604700BF53B9000001B40248844601BC29
:103FA000604700BFA1AF000001B40248844601BCD5
:103FB000604700BF6D0B010001B40248844601BC9C
:103FC000604700BFC95C010001B40248844601BCDF
:103FD000604700BFF935010001B40248844601BCC6
:103FE000604700BF75A9000001B40248844601BCC7
:103FF000604700BF5976010001B40248844601BC05
:10400000604700BF4DF9000001B40248844601BC7E
:10401000604700BFF9ED000001B40248844601BCCE
:10402000604700BF1907010001B40248844601BC83
:10403000604700BFDD0C010001B40248844601BCAA
:10404000604700BF3D71010001B40248844601BCD5
:10405000604700BFBD0B010001B40248844601BCAB
:10406000604700BF8B52010001B40248844601BC86
:10407000604700BFEDA5000001B40248844601BCC2
:10408000604700BFA9D8000001B40248844601BCC3
:10409000604700BF6911010001B40248844601BCB9
:1040A000604700BF51B8000001B40248844601BC1B
:1040B000604700BFDD0A010001B40248844601BC2C
:1040C000604700BFB70E000001B40248844601BC3F
:1040D000604700BFE512010001B40248844601BCFC
:1040E000604700BFE9D4000001B40248844601BC27
:1040F000604700BFED68010001B40248844601BC7E
:10410000604700BFC115010001B40248844601BCEC
:10411000604700BFD544010001B40248844601BC99
:10412000604700BF0189000001B40248844601BC19
:10413000604700BFC1F7000001B40248844601BCDB
:10414000604700BF21A9000001B40248844601BCB9
:10415000604700BFE1AC000001B40248844601BCE6
:10416000604700BF016C010001B40248844601BCF5
:10417000604700BF6137010001B40248844601BCBA
:10418000604700BF090E000002000000967A02118D
:10419000010000000879021102000000927A021169
:1041A00001000000C841FF1F020000001079021149
:1041B00001000000E861FF1F02000000907A021178
:1041C00003000000BC61FF1F12000000020000009D
:1041D000967A0211010000007079021102000000BD
:1041E000927A021101000000A142FF1F02000000AC
:1041F00082790211010000006B79021102000000B7
:10420000927A021101000000A042FF1F020000008C
:104210008079021101000000CC61FF1F0200000044
:10422000927A0211010000009F42FF1F020000006D
:104230007E790211010000005B790211020000008A
:10424000927A0211010000009E42FF1F020000004E
:104250007C79021101000000567902110200000071
:10426000927A0211010000009D42FF1F020000002F
:104270007A79021101000000517902110200000058
:10428000927A0211010000009C42FF1F0200000010
:1042900078790211010000004C7902110202020239
:1042A00002020000B5080211B1080211867902115C
:1042B00090011D0018001800FFFF0701020304050C
:1042C00006020106000000000000000000000000DF
:1042D00000000000000000000000000000000000DE
:1042E0000300000002000000967A021101000000A5
:1042F000087A021102000000927A02110100000007
:104300005443FF1F02000000127A02110100000056
:10431000E261FF1F02000000907A0211030000001A
:104320002864FF1F02000000927A021101000000C1
:104330005443FF1F02000000107A02110100000028
:10434000E461FF1F02000000907A021103000000E8
:104350002064FF1F12000000010000009779021185
:104360000B000500F7000000B4000028002800281A
:104370003075A000A000A000A00000080008E00127
:10438000F00010001000100010001000100050008D
:104390005000500010001000D00700000000000086
:1043A0000F0001000500307507001000010081FFBB
:1043B00000000000FF000000A9290211B12702112E
:1043C00041250211FFFF0100FF000000A55302116B
:1043D00021510211395002110000000000000000BC
:1043E00000000800040000003B0001085902E00141
:1043F00088212800FF00000002000000967A0211C8
:10440000010000005C7B021102000000927A0211A0
:10441000010000007544FF1F020000008E7A0211A7
:10442000010000003468FF1F02000000927A0211B0
:10443000010000007444FF1F020000008C7A02118A
:10444000010000007244FF1F02000000927A021176
:10445000010000007044FF1F020000008A7A021170
:10446000010000006844FF1F180018001D009001A3
:10447000020000030202000002000000967A02110E
:1044800001000000707B021102000000927A02110C
:1044900001000000B844FF1F02000000887A0211EA
:1044A000000000000000000002000000907A0211ED
:0C44B000030000005468FF1F20FF000004
:040000051FFF184180
:00000001FF
